S01900006F70656E626C745F73746D3332683734332E73726563F9
S315080000000000082485090008990800089B080008CC
S315080000109D0800089F080008A108000800000000C5
S31508000020000000000000000000000000A30800080F
S31508000030A508000800000000A7080008A90800088D
S31508000040D5090008D5090008D5090008D50900080A
S31508000050D5090008D5090008D5090008D5090008FA
S31508000060D5090008D5090008D5090008D5090008EA
S31508000070D5090008D5090008D5090008D5090008DA
S31508000080D5090008D5090008D5090008D5090008CA
S31508000090D5090008D5090008D5090008D5090008BA
S315080000A0D5090008D5090008D5090008D5090008AA
S315080000B0D5090008D5090008D5090008D50900089A
S315080000C0D5090008D5090008D5090008D50900088A
S315080000D0D5090008D5090008D5090008D50900087A
S315080000E0D5090008D509000800000000D509000850
S315080000F0D5090008D5090008D5090008D50900085A
S31508000100D5090008D5090008D5090008D509000849
S31508000110D5090008D5090008D5090008D509000839
S31508000120D5090008D5090008D5090008D509000829
S31508000130D5090008D5090008D5090008D509000819
S3150800014000000000000000000000000000000000A1
S31508000150D5090008D5090008D5090008D5090008F9
S31508000160D5090008D5090008D5090008D5090008E9
S31508000170D5090008D5090008D509000800000000BF
S31508000180D5090008D5090008D5090008D5090008C9
S31508000190D5090008D5090008D5090008D5090008B9
S315080001A0D5090008D5090008D5090008D5090008A9
S315080001B0D5090008D5090008D5090008D509000899
S315080001C0D5090008D5090008D5090008D509000889
S315080001D0D5090008D5090008D5090008D509000879
S315080001E0D5090008D5090008D5090008D509000869
S315080001F0D5090008D5090008D5090008D509000859
S31508000200D5090008D5090008D5090008D509000848
S31508000210D5090008D5090008D5090008D509000838
S31508000220D5090008D5090008D5090008000000000E
S31508000230D5090008D509000800000000D5090008FE
S31508000240D5090008D5090008D5090008D509000808
S31508000250D5090008D5090008D5090008D5090008F8
S31508000260D5090008D5090008D5090008D5090008E8
S31508000270D5090008D5090008D509000800000000BE
S31508000280D5090008D5090008D509000800000000AE
S30D0800029000000000D509000872
S3150800029810B5054C237833B9044B13B10448AFF3AA
S315080002A800800123237010BDC80000240000000048
S315080002B8F061000808B5034B1BB103490348AFF3BF
S315080002C8008008BD00000000CC000024F06100088A
S315080002D808B505F051FA08BD08B505F05BFA08BD7A
S315080002E808B5054B1B6913F4005F01D0002008BD4B
S315080002F800F03EF80120FAE70008025808B564201D
S3150800030800F008F808BD08B500F00AF808BD7047F7
S3150800031870477047014B1880704700BFE4000024F7
S3150800032808B504F0E9FF0E4B1B6898420FD30D4B2E
S315080003381B786BB90B4B01221A700B4B80229A61FA
S3150800034804F0DAFF094B1B881844054B186008BDEA
S31508000358044B00221A70044B4FF400029A61EFE727
S31508000368E8000024E600002400040258E4000024FB
S31508000378024B4FF400029A61704700BF0004025806
S3150800038870B58CB000240794089409940A940B94C1
S315080003982B4BD3F8E02042F00402C3F8E020D3F848
S315080003A8E02002F004020592059AD3F8E02042F00C
S315080003B88002C3F8E020D3F8E02002F08002049215
S315080003C8049AD3F8E02042F00802C3F8E020D3F8EC
S315080003D8E02002F008020392039AD3F8E02042F0DC
S315080003E80102C3F8E020D3F8E02002F001020292E5
S315080003F8029AD3F8E02042F00202C3F8E020D3F8C4
S31508000408E03003F002030193019B0E4E4FF40003FC
S31508000418B3610CAD4FF4005345F8183D29460A4810
S3150800042802F026FC8023069301230793089409946F
S315080004380A942946304602F01BFC0CB070BD00BF72
S3150800044800440258000402580008025810B590B033
S31508000458202200210DEB020005F0BDFE00240494BD
S31508000468059406942B4BD3F8E82042F48022C3F867
S31508000478E820D3F8E82002F480220192019AD3F8FA
S31508000488E02042F00802C3F8E020D3F8E03003F091
S3150800049808030093009B4FF44073029302230393C7
S315080004A80723079302A91C4802F0E2FB08944FF4B5
S315080004B8E13309930A940B940C940C230D930E9428
S315080004C80F94164C08A9204602F07AFFA36823F071
S315080004D86043A360A36823F06063A360236823F0DE
S315080004E800532360636823F490436360A36823F08A
S315080004F82A03A360236843F001032360074BDB69DB
S3150800050813F4001FFAD0054BDB6913F4800FF5D0F6
S3150800051810B010BD00440258000C025800480040AC
S3150800052810B5564A136823F00F0343F00403136003
S31508000538524B1B6803F00F03042BF9D1504AD368B2
S3150800054823F0070343F00203D360936943F4404357
S3150800055893614C4B1A6842F480221A601A6842F46E
S3150800056880321A60474B1B6813F4003FFAD0454B94
S315080005789A6A22F0030242F002029A62DA6A42F49E
S315080005888032DA62DA6A42F40032DA62DA6A22F029
S315080005980C0242F00402DA62DA6A22F00202DA622D
S315080005A89A6A22F47C7242F040029A621A6B3649B9
S315080005B8114040F2DF120A431A631A6B22F47E428C
S315080005C842F400721A631A6B22F4FE0242F4981275
S315080005D81A631A6B22F0FE4242F080721A631A688E
S315080005E842F080721A60274B1B6813F0007FFAD016
S315080005F8244CA36923F00F0343F00803A361236976
S3150800060823F0070343F003032361A36923F4706304
S31508000618A361A36923F00F0343F00803A361E36901
S3150800062823F0700343F04003E361E36923F4E063CE
S3150800063843F48063E361A36923F0700343F040033E
S31508000648A361236A23F0700343F0400323620F482B
S3150800065803F0F4FC002000F0FDF90D4A136823F0B6
S3150800066807031360236D23F040532365636D23F452
S31508000678401343F48013636510BD00BF0020005281
S31508000688004802580044025800FEFFFF00389C1C28
S315080006985444025808B500F005FAFFF741FFFFF77A
S315080006A86FFEFFF7D3FEFFF713FEFFF715FEFCE70D
S315080006B882B0074BD3F8F42042F00202C3F8F420BC
S315080006C8D3F8F43003F002030193019B02B0704794
S315080006D80044025800B589B0002303930493059390
S315080006E8069307930268154B9A4202D009B05DF83B
S315080006F804FB134BD3F8EC2042F48072C3F8EC20C1
S31508000708D3F8EC2002F480720192019AD3F8E0201B
S3150800071842F00202C3F8E020D3F8E03003F00203FF
S315080007280293029B4FF4407303930223049309230D
S31508000738079303A9034801F0B7F8D7E700A00040D4
S31508000748004402580004025810B588B000230393E1
S3150800075804930593069307930268154B9A4201D0AA
S3150800076808B010BD134CD4F8E03043F00103C4F8C0
S31508000778E030D4F8E03003F001030193019B4FF40D
S31508000788C0530393022304930A23079303A90A4829
S3150800079801F08AF8D4F8D83043F00063C4F8D830A2
S315080007A8D4F8D83003F000630293029BD8E700BF59
S315080007B800000840004402580000025808B50268BC
S315080007C8084B9A4200D008BD074AD2F8D83023F019
S315080007D80063C2F8D8304FF4C051044801F054F900
S315080007E8F1E700BF0000084000440258000002581C
S315080007F810B502F0A3FA214C4FF40003A361204870
S3150800080802F04AF91F4802F047F9204602F044F96F
S315080008181D4802F041F91D4BD3F8D82022F0006292
S31508000828C3F8D820D3F8EC2022F48072C3F8EC2059
S31508000838D3F8E82022F48022C3F8E820D3F8E02089
S3150800084822F00802C3F8E020D3F8E02022F00402D8
S31508000858C3F8E020D3F8E02022F00202C3F8E0202B
S31508000868D3F8E02022F00102C3F8E020D3F8F420F8
S3150800087822F00202C3F8F42010BD00BF0004025893
S31508000888000C025800080258000002580044025892
S315080008987047FEE7FEE7FEE7FEE7704770477047D2
S315080008A808B500F02DF908BD294AD2F8883043F46E
S315080008B87003C2F88830274B1B6803F00F03062B12
S315080008C806D8244A136823F00F0343F00703136076
S315080008D8214B1A6842F001021A6000221A61196847
S315080008E81E4A0A401A601B4B1B6803F00F03072BA6
S315080008F806D9184A136823F00F0343F00703136051
S31508000908154B00229A61DA611A62154999621549E6
S31508000918D962154919635A639963DA6319645A647B
S31508000928196821F4802119601A66104B1A68104B49
S315080009381340B3F1005F02D20E4B01221A600E4B28
S3150800094843F2D2021A60024B4FF000629A6070476F
S3150800095800ED00E000200052004402587FEDF6EA58
S31508000968000202020000FF01800201010010005C7B
S315080009780000FFFF0881005100400052DFF834D01C
S31508000988FFF792FF002103E00B4B5B5843500431F5
S315080009980A480B4B42189A42F6D30A4A02E0002341
S315080009A842F8043B084B9A42F9D305F0E5FBFFF7F2
S315080009B871FE704700000824BC6400080000002483
S315080009C8C8000024C800002498150024FEE7000083
S315080009D810B5194B194ADA670024DC67184AC3F8B0
S315080009E88020C3F8804040F27122C3F88420C3F8F7
S315080009F88440144AC3F88820C3F888401822C3F8E4
S31508000A088C20C3F88C40104AC3F89020C3F890404D
S31508000A184FF49B72C3F89420C3F894400B4AC3F862
S31508000A289820C3F898400A4AC3F89C20C3F89C4003
S31508000A38FFF7DEFE204610BD00440258315001007B
S31508000A4823C0000AFF072803FFC3FFE83330D7315E
S31508000A58AADE2000104B1B780BB90120704710B589
S31508000A6804464FF47A70B0FBF3F30C4A1068B0FBEF
S31508000A78F3F000F0A9F868B90F2C01D901200AE0AB
S31508000A88002221464FF0FF3000F06CF8044B1C603A
S31508000A98002000E0012010BD080000240000002402
S31508000AA80C00002410B5032000F04AF801F0DCFE1B
S31508000AB80F498B69C3F303230E4AD35C03F01F035C
S31508000AC8D8408B6903F00F03D35C03F01F0320FAA1
S31508000AD803F3094A1360094B18600020FFF7BAFFA9
S31508000AE810B10124204610BD0446FFF7E1FDF9E7D9
S31508000AF80044025854620008040000240000002438
S31508000B08034B1B78034A11680B441360704700BFF0
S31508000B18080000243813002438B5044604F0F4FB0A
S31508000B280546B4F1FF3F02D0044B1B781C4404F079
S31508000B38EBFB401BA042FAD338BD00BF08000024CF
S31508000B480649CB6823F4E0631B041B0C000200F477
S31508000B58E0600343024A1A43CA60704700ED00E0A2
S31508000B680000FA0530B4154BDB68C3F30223C3F15A
S31508000B780704042C28BF04241D1D062D14D9033B7D
S31508000B884FF0FF3505FA04F421EA0401994005FAFD
S31508000B9803F322EA03031943002807DB0901C9B24C
S31508000BA8074B195430BC70470023E9E700F00F00DB
S31508000BB80901C9B2034B1954F4E700BF00ED00E078
S31508000BC800E400E014ED00E00138B0F1807F0AD2B5
S31508000BD8064B5860064AF02182F8231000209860D0
S31508000BE807221A6070470120704700BF10E000E02E
S31508000BF800ED00E030B4446B0268D2F884106F4BFD
S31508000C08194041EA8401C2F884100268D2F88410AF
S31508000C1821F47F01856B41EA0541C2F88410826B8D
S31508000C2822440468D4F88810194041EA8201C4F8B5
S31508000C3888100468D4F8881021F4FE01C56B41EAC7
S31508000C480541C4F88810C16B02EB41020468D4F860
S31508000C58A010194041EA8201C4F8A0100468D4F823
S31508000C68A01021F4FE01056C41EA0541C4F8A0105C
S31508000C78046C416C01FB04240268D2F8B0101940D0
S31508000C8841EA8401C2F8B0100268D2F8B01021F41B
S31508000C98FE01856C41EA0541C2F8B010826CC16C48
S31508000CA801FB02440268D2F8AC10194041EA8401F3
S31508000CB8C2F8AC10026D416D01FB02420468D4F813
S31508000CC8F010194041EA8201C4F8F0100468D4F813
S31508000CD8F01021F47C11856D41EA0541C4F8F0103D
S31508000CE8816D02EB41020468D4F8C0100B4043EA50
S31508000CF88202C4F8C0200268D2F8C03023F47C13F4
S31508000D08C16D43EA0143C2F8C0300268D2F8C03060
S31508000D1823F07C53016E43EA0163C2F8C030436B83
S31508000D28274A1A449200C266836B02EB8303036759
S31508000D38C16B03EBC1034367046C416C01FB04F107
S31508000D4803EB81038367846CC16C01FB04F103EB35
S31508000D588103C367046D416D01FB04F103EB81034D
S31508000D68C0F88030816D03EBC103C0F88430C46DC8
S31508000D78856E05FB04F403EB8403C0F88830016E1E
S31508000D8801FB05F103EB8103C0F890300D498B424E
S31508000D980DD9D0F89C3043F02003C0F89C300323C3
S31508000DA880F89830012007E0002342F8043BD0F881
S31508000DB890309342F8D8002030BC70470300FFFFF4
S31508000DC8002B0010FCD30040F0B44C68E4B90E6957
S31508000DD88C6826430C6846EA84460D6ACC6944EA58
S31508000DE805648D692C434D692C43CD682C43D0F88E
S31508000DF88470806E03FB00F307EB830547F82360CE
S31508000E086C600835002015E00E698C6826430C6866
S31508000E18264346F08046E0E71418E678A3781B04CC
S31508000E2843EA0663647843EA0423145C234345F8D3
S31508000E38043B0430CB89034CE35C8342ECD8F0BC12
S31508000E48704700BF6462000830B595B004464C2266
S31508000E58A04901A805F0B4F9002C00F038812368E8
S31508000E689D4A934220D094F898300BB32268936928
S31508000E7823F01003936104F047FA054623689A6934
S31508000E8812F0080F1AD004F03FFA401B0A28F5D9C1
S31508000E98D4F89C3043F00103C4F89C30032384F843
S31508000EA89830012015B030BD03F580736360DAE722
S31508000EB884F899302046FFF70DFCD7E79A6942F07F
S31508000EC801029A6104F020FA054623689A6912F025
S31508000ED8010F0FD104F018FA401B0A28F5D9D4F8DF
S31508000EE89C3043F00103C4F89C30032384F89830F7
S31508000EF80120D7E79A6942F002029A61237C012BFE
S31508000F0840D02268936943F040039361637C012BC0
S31508000F183ED02268936923F480439361A37C012B0E
S31508000F283CD02268936943F4805393612268936995
S31508000F3823F44073A1680B4393612268936923F0ED
S31508000F48A40393612268136923F010031361E36805
S31508000F58012B29D0002B2CD0022B00F09B8022686D
S31508000F68936943F0800393612268136943F0100379
S31508000F781361E368032B1CD12268936943F02003A5
S31508000F88936116E02268936923F040039361BDE7ED
S31508000F982268936943F480439361BFE7226893699B
S31508000FA823F480539361C1E72268936943F00403E5
S31508000FB89361A3695A1EE369013B1B0243EA42632C
S31508000FC8226A013A13436269013A216843EA0243ED
S31508000FD8CB61A368B3F5407F62D0236E33B122682C
S31508000FE8D2F8C030616E0B43C2F8C030E36D226E8A
S31508000FF8D3420DD02168D1F8C83023F00703A26E72
S3150800100814A800EB820252F84C2C1343C1F8C830D6
S31508001018236C6BB12168D1F8BC3023F00703626CE6
S3150800102814A800EB820252F84C2C1343C1F8BC30C2
S31508001038A36C73B12168D1F8BC3023F07003E26C55
S3150800104814A800EB820252F84C2C43EA0213C1F8A2
S31508001058BC30236D73B12168D1F8BC3023F4E06342
S31508001068626D14A800EB820252F84C2C43EA02235C
S31508001078C1F8BC302268184B9A4222D00023C4F81B
S315080010889430C4F89C30012384F898302046FFF73A
S31508001098B1FD07E72268936943F02003936188E75F
S315080010A8A36A013BE26A013A43EA0223226B013A40
S315080010B843EA0213626A013A216843EA0243CB60AB
S315080010C88BE76268936823F003039360D6E70120E9
S315080010D8E8E600BF0862000800A0004090F89830CB
S315080010E8013BDBB2012B07D9D0F89C3043F0020349
S315080010F8C0F89C3001207047CB680A68D2B9072B1C
S315080011080ED08A68DB0643EA82730A6943EA024311
S315080011184A691343C26E496842F82130002070476D
S315080011280A69CB691B0243EA02438A69134343F0F7
S315080011386053EFE710B40A6942EA4372072B0ED0E8
S315080011488C684B6943EA8473006F496800EBC104ED
S3150800115840F83120636000205DF8044B70478B69BE
S31508001168F2E710B490F89840E4B2012C09D0D0F808
S315080011789C3043F00403C0F89C3001205DF8044B0A
S315080011887047920042EA011141EA4303026801994D
S315080011980B43C2F880300020F0E790F89830DBB2AD
S315080011A8012B07D0D0F89C3043F00403C0F89C30D4
S315080011B801207047022380F898300268936923F063
S315080011C8010393610023C0F89C301846704770B530
S315080011D890F89840013CE4B2012C07D9D0F89C3025
S315080011E843F00203C0F89C30012070BD93FAA3F5BA
S315080011F8B5FA85F50668D6F8C040C4F30544A5428D
S315080012080BD2D6F8CC401C420FD0D0F89C3043F00D
S315080012184003C0F89C300120E7E7D0F89C3043F03B
S315080012282003C0F89C300120DFE793FAA3F3B3FA4A
S3150800123883F3FFF7C9FD0020D7E790F89830DBB2AB
S31508001248022B07D0D0F89C3043F00803C0F89C302E
S31508001258012070470368C3F8D010002070470000C3
S31508001268F0B490F89840E4B2022C08D0D0F89C3034
S3150800127843F00803C0F89C300120F0BC70474029A9
S3150800128839D0412964D0046D8C4240F28E80C46FEF
S31508001298456D01FB05F504EB85044FF0000C256840
S315080012A805F080455560002D40F087802568C5F310
S315080012B88A451560256805F000559560256805F086
S315080012C800451561A588D561656805F47025D5605A
S315080012D8656805F480155561656805F40015956116
S315080012E8E57905F07F0515626568ED0F556204F125
S315080012F80805002469E00468D4F8A05015F4FE0F20
S3150800130816D0D4F8A45015F07F0F19D0D4F8A450E5
S3150800131815F0807F01D0D4F8A050D4F8A440C4F3BF
S31508001328052C446F456C0CFB05F504EB8504B6E7FC
S31508001338D0F89C3043F02003C0F89C3001209CE785
S31508001348D0F89C3043F48073C0F89C30012094E7A9
S315080013580468D4F8B05015F4FE0F16D0D4F8B45073
S3150800136815F07F0F19D0D4F8B45015F0807F01D046
S31508001378D4F8B050D4F8B440C4F3052C846FC56CBF
S315080013880CFB05F504EB850489E7D0F89C3043F097
S315080013982003C0F89C3001206FE7D0F89C3043F44E
S315080013A88073C0F89C30012067E7D0F89C3043F07A
S315080013B82003C0F89C3001205FE7256825F06045C2
S315080013C8156077E72E5D1E550134D689124FBE5D26
S315080013D8A642F7D840290BD041290ED01F2911D883
S315080013E80268012303FA01F1C2F89810002044E7BD
S315080013F80368C3F8A8C000203FE70368C3F8B8C065
S3150800140800203AE701F01F010268012303FA01F1F7
S31508001418C2F89C10002030E7646200080368D3F815
S31508001428CC300B4201D00120704700207047402974
S3150800143805D00368D3F8B40000F07F007047036846
S31508001448D3F8A40000F07F0070470000144BDB684F
S3150800145813F0010F09D0124B124A5A6002F188326A
S315080014685A60DB6813F0010F16D10D4BD3F80C310F
S3150800147813F0010F12D00A4B0A4AC3F8042102F1E5
S315080014888832C3F80421D3F80C3113F0010F01D1BF
S3150800149800207047012070470120704700207047D8
S315080014A800200052230167450D4BDA6842F0010215
S315080014B8DA60DB6813F0010F0FD0094BD3F80C215B
S315080014C842F00102C3F80C21D3F80C3113F0010FCE
S315080014D801D000207047012070470120704700BFDF
S315080014E8002000522DE9F04105460F46384B1E6983
S315080014F803F00AFF8046022F07D026F0684626F42E
S315080015088016760C7604042420E0314BD3F8106153
S3150800151826F0684626F48016760C760446F00046C9
S315080015282C4C13E003F0F0FEA0EB0800A84248D8BC
S3150800153865B9032025E0264B1B6934EA03030CBF6B
S315080015480123002383B1B5F1FF3FEBD134F004033F
S31508001558F1D01F4BD3F8103124EA030333F00043C4
S315080015680CBF01230023EDE736F000410FD01A4AD5
S31508001578936933439361002E05DA154BC3F81411A2
S315080015880120BDE8F081124B5E610120F9E7012FC1
S315080015980CD00F4BD3F8103113F4803F15D00C4BF1
S315080015A84FF48032C3F814210020EAE7084B1B6978
S315080015B813F4803F07D0064B4FF480325A61002057
S315080015C8DFE70320DDE70020DBE70020D9E700BFD7
S315080015D800200052040000803C1300242F4B1B7D7A
S315080015E8012B56D070B50C4615462C4B01221A7598
S315080015F801F17843B3F5801F3DD3A1F10161B1F537
S31508001608801F49D20226254B00229A6131464CF2A0
S315080016185030FFF767FF034640BB012E2DD0204AFE
S31508001628D2F80C3143F00203C2F80C31BFF36F8FBE
S31508001638BFF34F8F082355F8042B44F8042B013BB6
S3150800164813F0FF03F7D1BFF36F8FBFF34F8F314600
S315080016584CF25030FFF746FF0346012E13D01049C7
S31508001668D1F80C2122F00202C1F80C210B4A0021FC
S315080016781175184670BD0126C5E7094AD36843F0AF
S315080016880203D360D2E70649CA6822F00202CA6092
S31508001698ECE70223184670470123EAE73C130024BF
S315080016A80020005201F00303032B24D011F0010F88
S315080016B80BD01D4BDA6822F03002DA60DA6802438A
S315080016C8DA60DA6842F08802DA6011F0020F11D09F
S315080016D8154BD3F80C2122F03002C3F80C21D3F8A5
S315080016E80C211043C3F80C01D3F80C2142F08802E8
S315080016F8C3F80C2170470C4BDA6822F03002DA601E
S31508001708D3F80C2122F03002C3F80C21DA68024318
S31508001718DA60D3F80C211043C3F80C019A6942F031
S3150800172810029A61704700BF0020005230B411F0C9
S31508001738010F0BD0104CE36823F4E663E360E36813
S3150800174842EA00252B4343F08403E36011F0020FB5
S315080017580FD00949D1F80C3123F4E663C1F80C31E6
S31508001768D1F80C3142EA00221A4342F08402C1F841
S315080017780C2130BC704700BF00200052F8B5474B13
S315080017881B7D012B00F088800F460446434B012237
S315080017981A7500229A61436813F0010F0DD10026C5
S315080017A8636813F0020F12D1CEB92368012B1BD038
S315080017B84FF0FF333B60A5684CE001214CF25030EE
S315080017C8FFF790FE06460028EAD00126E8E7022138
S315080017D84CF25030FFF786FE0028E5D001262F4B3D
S315080017E800221A753046F8BD61682069FFF75AFF66
S315080017F8636813F0010F12D1636813F0020FEED075
S3150800180802214CF25030FFF76DFE00B10126244A3A
S31508001818D2F80C3123F00803C2F80C31DFE70121AE
S315080018284CF25030FFF75EFE00B101261C4AD36819
S3150800183823F00803D360DFE701214CF25030FFF7A5
S3150800184851FE0646164AD168164B0B40D3600FE080
S3150800185806BB0135E368A2681344AB42BFD92269BF
S3150800186861682846FFF762FF636813F0010FE3D142
S31508001878636813F0020FEBD002214CF25030FFF7E1
S3150800188831FE0646064AD2F80C11064B0B40C2F83A
S315080018980C31DDE73D60A2E70226A3E73C130024E6
S315080018A800200052FBF8FFFFF0B583B000233AE0AA
S315080018B8092400E00024B4403C4302356E4E46F83D
S315080018C825406E4C2568D44304EA05064F6817F484
S315080018D8803F01D042EA0506684D2E606E6804EA24
S315080018E806054F6817F4003F01D042EA0605634E1D
S315080018F875604FF0B0452D6804EA05064F6817F479
S31508001908801F01D042EA05064FF0B0452E606D6883
S315080019182C404E6816F4001F01D042EA05044FF021
S31508001928B042546001330A6832FA03F400F0A28020
S3150800193801249C402240F5D04D686E1E112D18BF13
S31508001948012E01D9122D12D186685F000325BD40E4
S3150800195826EA0506CD68BD4035438560466826EA09
S3150800196804064D68C5F300149C4034434460C668B1
S315080019785F000325BD40EC4326408D68BD403543CE
S31508001988C5604D68122D18BF022D13D1DE0808361A
S3150800199850F826E003F007054FEA850C0F2505FAE7
S315080019A80CF52EEA050E0D6905FA0CF545EA0E053D
S315080019B840F82650056825404C6804F00304BC40E6
S315080019C82C4304604C6814F0805FABD02C4CD4F8D8
S315080019D8F45045F00205C4F8F450D4F8F44004F07D
S315080019E802040194019C9D08AE1C234C54F82670E9
S315080019F803F00304A6000F24B44027EA0407214C81
S31508001A08A0423FF457AF04F58064A04222D004F5FB
S31508001A188064A04220D004F58064A0421ED004F554
S31508001A288064A0421CD004F58064A0421AD004F54C
S31508001A388064A04218D004F58064A04216D004F544
S31508001A488064A04214D004F58064A0423FF430AF05
S31508001A580A2430E701242EE702242CE703242AE780
S31508001A68042428E7052426E7062424E7072422E78A
S31508001A78082420E703B0F0BD000400588000005889
S31508001A880044025800000258002331FA03F200F015
S31508001A989880F0B52CE0092700E0002707FA04F437
S31508001AA8B44273D005685C00032606FA04F4254395
S31508001AB8056023FA06F5083550F8256003F0070788
S31508001AC84FEA870C0F2707FA0CF726EA070640F8A5
S31508001AD82560C568E4432540C560456825EA0202CD
S31508001AE84260826814408460013331FA03F267D091
S31508001AF801229A4012EA0105F6D04FEA930E0EF132
S31508001B080206304C54F8266003F00304A4004FF08C
S31508001B180F0C0CFA04FC0CEA06062B4FB842BCD08C
S31508001B2807F58067B84221D007F58067B8421FD005
S31508001B3807F58067B8421DD007F58067B8421BD0FD
S31508001B4807F58067B84219D007F58067B84217D0F5
S31508001B5807F58067B84215D007F58067B84213D0ED
S31508001B6807F58067B84296D00A2797E7012795E7C9
S31508001B78022793E7032791E704278FE705278DE7C9
S31508001B8806278BE7072789E7082787E70F4C26687C
S31508001B98ED432E40266066682E4066604FF0B044D6
S31508001BA826682E402660666835406560054E0EF143
S31508001BB8020456F8245025EA0C0546F8245071E71D
S31508001BC8F0BD70470004005800000258800000580D
S31508001BD82DE9F04782B00768CA00521A93000344F1
S31508001BE85A6D1B6D9A4257D8B8469B1AC1EBC10461
S31508001BF8A2000244526C9A4200D31A460C4606467C
S31508001C0802F1030A4FEA9A0A16E009F1030A4FEAAB
S31508001C189A0AE3001B1B9D003544A96C337C009384
S31508001C281FFA89F3E2B2384601F0B8FFAB6C4B44A9
S31508001C38AB646B6D4B446B6508EB441303F5106393
S31508001C489B699BB2534513D3E3001B1B9A00324486
S31508001C58516D136D99420BD253B15B1AC4EBC4018B
S31508001C688A003244D2F844909945CED39946CCE7AF
S31508001C78E3001B1B98000644326D736D9A420FD811
S31508001C8804F00F040121A140D7F8344824EA0104D6
S31508001C98C7F83448002000E0012002B0BDE8F08704
S31508001CA80020FAE7F0B58BB0002800F091800446CA
S31508001CB8056890F8BD3323B3032384F8BD33EB6B6B
S31508001CC813F4807F01D100232361206801F004FD05
S31508001CD8254655F8107B6E460FCD0FC60FCD0FC695
S31508001CE895E8030086E80300231D0ECB384601F065
S31508001CF831FC58B1022384F8BD33012528460BB0B8
S31508001D08F0BD80F8BC33FEF71FFDD5E70021206833
S31508001D1801F0E8FC002315E0D900C81A820022441D
S31508001D28012082F83D0082F83C30A2F842300020B3
S31508001D3882F83F0050649064CA1A910021440865E5
S31508001D480133DBB26568AB42E6D3002315E0D80059
S31508001D58C11A8A002244002182F8FD1182F8FC3152
S31508001D6882F8FF11C2F80412C2F80812C21A9000C3
S31508001D782044C0F810120133DBB29D42E7D8254645
S31508001D8855F8107B6E460FCD0FC60FCD0FC695E8D2
S31508001D98030086E80300231D0ECB384601F0E8FC4D
S31508001DA8054660B9002384F83830012384F8BD3322
S31508001DB8636A012B08D0206802F0BFF89EE7022361
S31508001DC884F8BD33012599E7204600F02FFDF2E790
S31508001DD8012593E7026890F8BC33012B19D010B592
S31508001DE8012380F8BC33836A012B0AD004460068AD
S31508001DF802F097F8206801F069FC002084F8BC0313
S31508001E0810BD8369012BF1D0936B43F48033936338
S31508001E18ECE70220704738B590F8BC33012B18D088
S31508001E280446012380F8BC33006801F055FC206895
S31508001E3802F043F8054628B1002384F8BC33012587
S31508001E48284638BD206802F078F8002384F8BC33A1
S31508001E58F6E70225F4E768B110B50446032380F8C7
S31508001E68BD33FFF7D8FF2046FEF7A8FC002084F804
S31508001E78BD0310BD0120704770B504460D460068BD
S31508001E88066C00EB411303F530639A68216901294A
S31508001E9811D037498E4254D03DB9C5EBC5029300D7
S31508001EA82344D3F81032002B5CD0E9B2204604F05C
S31508001EB831F8002070BD12F0080F09D02D498E425E
S31508001EC8F7D912F4004FF4D04FF400429A60F0E7BD
S31508001ED812F0200F28D112F0280FEAD125498E4290
S31508001EE802D912F4004F22D1E900491B8A0022447C
S31508001EF8D2F804121B69C3F31203C91AC2F81412DA
S31508001F08D2F80412D2F808320B44C2F8083235B9A6
S31508001F18C5EBC50293002344D3F810325BB1E9B286
S31508001F28204603F0F7FFC4E720229A60C1E74FF47A
S31508001F3800429A60BDE704F57172012102F04EF875
S31508001F48EDE712F4004F09D112F0200F01D0202234
S31508001F589A60E9B2204603F0DDFFAAE74FF400428B
S31508001F689A60A6E704F57172002102F037F89CE733
S31508001F780A31544F0A30544F38B5044603681D6C65
S31508001F8803EB4111D1F8082B0E4B9D4207D901F5F1
S31508001F98306112F4004F02D04FF400438B6020469C
S31508001FA803F0B0FF074B9D4202D92369012B01D0E4
S31508001FB8002038BD04F571720121206802F00EF878
S31508001FC8F6E700BF0A30544F2DE9F84F044605686E
S31508001FD8284601F0EFFF08B1BDE8F88F2F460646F8
S31508001FE8206801F0B6FF0028F6D0206801F0B1FF96
S31508001FF810F0020F04D02268536903F002035361F4
S31508002008206801F0A6FF10F0100F15D02268936912
S3150800201823F010039361D5F8208008F00F09C8F358
S315080020284343022B00F08580062B00F0A580226822
S31508002038936943F010039361206801F08AFF10F44E
S31508002048002F40F0AD80206801F083FF10F4802F40
S3150800205840F0F180206801F07CFF0028C0F25F811B
S31508002068206801F076FF10F4006F0AD0D5F8083812
S3150800207813F0010F40F06D812268536903F4006379
S315080020885361206801F065FF10F0006F15D02268CB
S31508002098536903F00063536194F8F433002B40F056
S315080020A85C81012184F8F41323685B6DC3F3830309
S315080020B8C4F8F833204600F0CDFB206801F049FF44
S315080020C810F4805F40F04D81206801F042FF10F45B
S315080020D8005F40F0AB81206801F03BFF10F0080F65
S315080020E840F0BC81206801F034FF10F4801F40F0EE
S315080020F8BE81206801F02DFF10F4001F40F0C18151
S31508002108206801F026FF10F0804F40F0C48120684F
S3150800211801F01FFF10F0040F3FF45EAF23685D68F7
S3150800212815F0040F40F0C081226853682B435360AA
S3150800213852E747F6F07318EA030F3FF478AF4FEA09
S31508002148C90BABEB09034FEA830AA2444FEA1818EE
S31508002158C8F30A02DAF80812284601F03FFEC8F35F
S315080021680A08DAF808324344CAF80832DAF81432A0
S315080021784344CAF814325AE7082204F57171284606
S3150800218801F02CFEC8F30A184FEAC903A3EB0901A4
S315080021988A002244D2F814324344C2F8143246E775
S315080021A8206801F0DAFE8046B14617E007EB4913C6
S315080021B80122C3F8082B49462046FFF75DFE1DE0B5
S315080021C807EB49130822C3F8082B49462046FFF7A8
S315080021D8D3FE16E009F101094FEA5808B8F1000FCD
S315080021E83FF431AF18F0010FF4D05FFA89F120688F
S315080021F801F0C3FE824610F0010FD7D11AF0080F76
S31508002208DED11AF0100F04D007EB49131022C3F8D1
S31508002218082B1AF0200F04D007EB49132022C3F81D
S31508002228082B1AF4005FD5D007EB49134FF4005270
S31508002238C3F8082BCEE7206801F097FE8046B1461A
S315080022482AE05946204603F071FE1AF0080F04D012
S3150800225807EB49130822C3F808291AF0100F04D007
S3150800226807EB49131022C3F808291AF0400F04D0BF
S3150800227807EB49134022C3F808291AF0020F04D0BD
S3150800228807EB49130222C3F808291AF0800F41D12F
S3150800229809F101094FEA5808B8F1000F3FF4DAAE18
S315080022A818F0010FF4D05FFA89FB5946206801F047
S315080022B86DFE824610F0010FC7D009F00F03012101
S315080022C801FA03F2D7F8343823EA0203C7F8343890
S315080022D807EB4913C3F8081923698B42B1D14FEAAA
S315080022E8C902A2EB090293002344596C9A6C0A4462
S315080022F89A64B9F1000FA4D1C9EBC9029300234423
S315080023081B6D002B9DD104F571720121206801F01F
S3150800231865FE96E749462046FFF75AFCB8E7D5F81A
S31508002328043823F00103C5F8043894F8F433012B6C
S3150800233808D0204603F040FE2268536903F000439C
S3150800234853618DE6002184F8F413204600F082FADA
S31508002358F2E7204603F016FE8EE6204603F012FE44
S31508002368ABE605F50068D8F8043023F00103C8F889
S3150800237804301021206801F0CDF920E007EB461358
S315080023884FF67F31C3F80819D3F8002922F400124A
S31508002398C3F80029D3F8002942F00062C3F80029D7
S315080023A8C3F8081BD3F8002B22F40012C3F8002B35
S315080023B8D3F8002B42F00062C3F8002B0136636895
S315080023C8B342DBD8D8F81C3043F00113C8F81C30E0
S315080023D8236BEBB1D8F8843043F00B03C8F8843084
S315080023E8D8F8443043F00B03C8F84430D5F8003819
S315080023F823F4FE63C5F8003804F57172217C206859
S3150800240801F0ECFD2268536903F4805353615BE6D7
S31508002418D8F8142042F22B031343C8F81430D8F816
S31508002428103043F00B03C8F81030DFE7206801F0D6
S31508002438C5FD206801F060FAE060256800F00AFB2F
S31508002448227B0146284601F0CBF8204603F080FD9A
S315080024582268536903F4005353613CE6204603F0A7
S3150800246870FD2268536903F0080353613AE60021B0
S31508002478204603F0B0FD2268536903F480135361BC
S3150800248837E60021204603F0A0FD2268536903F4C5
S315080024980013536134E6204603F0A3FD2268536906
S315080024A803F08043536132E6204603F0A4FD3BE679
S315080024B8026890F8BC33012B16D010B5012380F8B2
S315080024C8BC33836A012B07D00446006801F029FD4E
S315080024D8002084F8BC0310BD8369012BF4D0936BE4
S315080024E843F480339363EFE70220704790F8BC33D0
S315080024F8012B0BD010B50446012380F8BC330068BD
S3150800250801F01BFD002084F8BC0310BD02207047AB
S3150800251890F8BC33012B0DD010B50446012380F87A
S31508002528BC3380F83810006801F0EBFC002084F80A
S31508002538BC0310BD02207047F8B511F0800F28D1EA
S3150800254801F00F06F500AF1BBC00274604F5FC741E
S31508002558044404343E460644002586F8FD5101F035
S315080025680F012170A260E370627802B1E180022B44
S315080025781ED090F8BC33012B1DD00546012380F8E0
S31508002588BC332146006801F0C7F9002085F8BC036A
S31508002598F8BD01F00F06F500AF1BBC002746383416
S315080025A8044404343E460644012586F83D50D6E7D9
S315080025B800232371DDE70220EAE738B511F0800F1A
S315080025C821D101F00F05EA00541BA3001C4603F5A8
S315080025D8FC730344043325460544002285F8FD2187
S315080025E801F00F01197090F8BC23012A1AD0044685
S315080025F8012280F8BC231946006801F0D5F90020A5
S3150800260884F8BC0338BD01F00F04E200151BAB00C3
S315080026181D463833034404332C460444012284F8FF
S315080026283D20DDE70220EDE770B501F00F05EE0065
S31508002638711B8C0004F5FC740444211D761BB40038
S315080026480444C4F80822C4F810320023C4F8143223
S3150800265884F8FD3184F8FC510369012B06D065B16D
S31508002668DAB2006801F0AEFA002070BDC5EBC506FF
S31508002678B4000444C4F80C22F1E7DAB2006801F0A1
S3150800268801FAF1E701F00F01C1EBC1018B0018440B
S31508002698D0F81402704770B501F00F05EE00711BEB
S315080026A88C0038340444211D761BB4000444A26403
S315080026B8236500236365012384F83D3084F83C507C
S315080026C80369012B06D05DB1DAB2006801F07AFA1F
S315080026D8002070BDC5EBC506B4000444E264F2E701
S315080026E8DAB2006801F0CEF9F2E738B501F00F055D
S315080026F843689D4236D811F0800F20D1CA00541A73
S31508002708A3001C4603F5FC7303440433224602441B
S31508002718002182F8FD1101229A701D7090F8BC23D9
S31508002728012A21D00446012280F8BC2319460068EC
S3150800273801F068FB7DB1002084F8BC0313E0EA00C9
S31508002748511B8B00194638330344043301440122CC
S3150800275881F83D20DFE704F57172217C206801F0D5
S315080027683DFCE8E7012038BD0220FCE710B501F07A
S315080027780F0443689C422CD811F0800F1DD1E30042
S315080027881A1B91000A4601F5FC71014404310244FA
S31508002798002382F8FD3100238B700C7090F8BC3347
S315080027A8012B18D00446012380F8BC33006801F0D1
S315080027B856FB002084F8BC030CE0E3001A1B9100C2
S315080027C80A463831014404310244012382F83D306F
S315080027D8E1E7012010BD0220FCE730B40468606A0E
S315080027E829B10D46A36A00EB134000230CE040EA22
S315080027F80240A06212E003F1400104EB8101496836
S3150800280800EB11400133DBB2691E8B42F3D340EA71
S31508002818024005F13F0104EB81014860002030BC05
S31508002828704703685962002070470000024603682B
S315080028380121C0F8FC13002082F8F4039A6942F0D3
S3150800284800629A61596D024A0A435A65704700BF81
S315080028580300001070470000024AD36843F08073EB
S31508002868D360704700480258724B1B6903F0380357
S31508002878102B00F0DB80182B10D00BB16E48704770
S315080028886C4B1B6813F0200F00F0D280694B186850
S31508002898C0F3C100694B23FA00F07047654A916A8C
S315080028A801F00301906AC0F30510D36A03F0010327
S315080028B8526BC2F3CC0203FB02F307EE903AF8EE2A
S315080028C8677A002800F0B580012966D0F9B102298F
S315080028D800F08F8007EE100AF8EE476A9FED586AEF
S315080028E886EE267A534B1B6BC3F3080306EE903A1B
S315080028F8F8EE666A9FED536A67EE867A76EEA77AE9
S31508002908F7EE006A77EEA67A27EE277A61E0494B52
S315080029181B6813F0200F23D046490A68C2F3C10280
S31508002928464BD34007EE103AF8EE476A07EE100A08
S31508002938B8EE476A86EE867A0B6BC3F3080306EE8B
S31508002948903AF8EE666A9FED3F6A67EE867A76EE03
S31508002958A77AF7EE006A77EEA67A27EE277A38E09E
S3150800296807EE100AF8EE476A9FED376A86EE267A6A
S31508002978304B1B6BC3F3080306EE903AF8EE666A0B
S315080029889FED306A67EE867A76EEA77AF7EE006AE2
S3150800299877EEA67A27EE277A1BE007EE100AF8EEF6
S315080029A8476A9FED276A86EE267A224B1B6BC3F386
S315080029B8080306EE903AF8EE666A9FED226A67EE15
S315080029C8867A76EEA77AF7EE006A77EEA67A27EE83
S315080029D8277A184B1B6BC3F34623013307EE903A45
S315080029E8F8EE677AC7EE276AFCEEE67A17EE900ADB
S315080029F8704707EE100AF8EE476A9FED146A86EEE6
S31508002A08267A0C4B1B6BC3F3080306EE903AF8EECE
S31508002A18666A9FED0C6A67EE867A76EEA77AF7EE0F
S31508002A28006A77EEA67A27EE277AD2E7084870472B
S31508002A38024870470044025800093D000090D00338
S31508002A480024744A000000390024744C0024F44A0F
S31508002A5800127A0008B5FFF707FF0B4A9369C3F314
S31508002A6803230A49CB5C03F01F0320FA03F3926990
S31508002A7802F00F02885C00F01F0023FA00F0044AEF
S31508002A881060044A136008BD0044025854620008DE
S31508002A9804000024000000246A4B984222D06A4B9E
S31508002AA898422FD0694B98423CD0694B984249D0F6
S31508002AB8684B984256D0684B984263D0674B984201
S31508002AC870D0674B98427DD0664B984200F08A8052
S31508002AD8654B984200F09680644B984200F0A280B5
S31508002AE80120704703F58843D3F8882042F001028D
S31508002AF8C3F88820D3F8882022F00102C3F8882072
S31508002B080020704703F58043D3F8882042F0020274
S31508002B18C3F88820D3F8882022F00202C3F8882050
S31508002B280020704703F57053D3F8882042F0040252
S31508002B38C3F88820D3F8882022F00402C3F888202E
S31508002B480020704703F56053D3F8882042F008023E
S31508002B58C3F88820D3F8882022F00802C3F888200A
S31508002B680020704703F55053D3F8882042F0100226
S31508002B78C3F88820D3F8882022F01002C3F88820E2
S31508002B880020704703F54053D3F8882042F0200206
S31508002B98C3F88820D3F8882022F02002C3F88820B2
S31508002BA80020704703F53053D3F8882042F04002D6
S31508002BB8C3F88820D3F8882022F04002C3F8882072
S31508002BC80020704703F52053D3F8882042F0800286
S31508002BD8C3F88820D3F8882022F08002C3F8882012
S31508002BE80020704703F51053D3F8882042F4807202
S31508002BF8C3F88820D3F8882022F48072C3F888207E
S31508002C080020704703F50053D3F8882042F4007271
S31508002C18C3F88820D3F8882022F40072C3F88820DD
S31508002C280020704703F5E053D3F8882042F4806201
S31508002C38C3F88820D3F8882022F48062C3F888204D
S31508002C48002070470000025800040258000802587D
S31508002C58000C0258001002580014025800180258AE
S31508002C68001C02580020025800240258002802585E
S31508002C78F0B40A6892FAA2F2B2FA82F216E00F697A
S31508002C88C66803FB03F505EB4504E443264005FB44
S31508002C9807F73E43C6604E68022E29D04B68066879
S31508002CA8344005FB03F32343036001320B6833FA08
S31508002CB802F440D0012494402340F6D04C68013CE5
S31508002CC8012CDCD88E68846803FB03F505EB4507F9
S31508002CD824EA070405FB06F52C4384600E68CD68CC
S31508002CE8446824EA060405FB06F52C434460C6E74F
S31508002CF8FF2B0ED8066A05FB03F707FB03F3C3EB9E
S31508002D08031726EA07074E6903FB06F33B430362E4
S31508002D18C4E7466A1B0A03FB03F707FB03F707FB27
S31508002D2803F3C3EB031726EA07074E6903FB06F303
S31508002D383B434362B2E70020F0BC70472D4B1B6843
S31508002D4803F00F03062B06D82A4A136823F00F0345
S31508002D5843F007031360284A136843F00103136016
S31508002D68254B1B6813F0040FFAD0234B00221A616F
S31508002D781968224A0A401A601F4B1B6813F0007F1D
S31508002D88FAD11D4B1B6813F0006FFAD11A4B1B6852
S31508002D9813F0005FFAD1184B00229A61DA611A62B9
S31508002DA8174999621749D962174919635A63996382
S31508002DB8DA6319645A64196821F4802119601A6655
S31508002DC8996E40F2FF720A439A66D3F8D02042F405
S31508002DD88032C3F8D020074B1B6803F00F03072B74
S31508002DE806D9044A136823F00F0343F00703136050
S31508002DF8704700BF002000520044025845EDF6EA25
S31508002E08000202020000FF018002010107EE900A93
S31508002E18F8EE676A07EE901AF8EE677A86EEA77AEA
S31508002E2807EE902AF8EE677A06EE903AF8EE666AA2
S31508002E389FED096A66EE866A77EEA67A27EE277AFE
S31508002E48DDED007AF8EE677AC7EE276AFCEEE67AD1
S31508002E5817EE900A704700BF000000392DE9F041C7
S31508002E6882B03F4B9B6A03F00303012B60D0002B0B
S31508002E7852D0022B63D00027002303604360836087
S31508002E88374B9E6AC6F305161A6BC2F30802551C19
S31508002E98DB6A13F0010F5FD0314B5B6BC3F3CC08C9
S31508002EA8002E36D004462E4BDB6A13F4803F0CD02E
S31508002EB82B4B1B6BC3F346230133009343462A4621
S31508002EC831463846FFF7A2FF2060254BDB6A13F424
S31508002ED8003F0CD0224B1B6BC3F306430133009308
S31508002EE843462A4631463846FFF790FF60601C4B32
S31508002EF8DB6A13F4802F0CD0194B1B6BC3F30663DC
S31508002F080133009343462A4631463846FFF77EFF83
S31508002F18A06002B0BDE8F081114B1B6813F0040FDE
S31508002F2814D00F4B1B68C3F3C1030E4FDF40A3E74A
S31508002F380B4B1B6813F4807F0AD100279CE7084BC4
S31508002F481B6813F4003F05D1002795E7002793E788
S31508002F58054F91E7054F8FE74FF00008A0E700BF38
S31508002F68004402580090D00300093D0000127A0078
S31508002F782DE9F04182B03F4B9B6A03F00303012B0E
S31508002F8860D0002B52D0022B63D0002700230360A1
S31508002F9843608360374B9E6AC6F305369A6BC2F35D
S31508002FA80802551CDB6A13F0100F5FD0314BDB6B38
S31508002FB8C3F3CC08002E36D004462E4BDB6A13F42E
S31508002FC8002F0CD02B4B9B6BC3F34623013300937E
S31508002FD843462A4631463846FFF718FF2060254BF0
S31508002FE8DB6A13F4801F0CD0224B9B6BC3F3064392
S31508002FF80133009343462A4631463846FFF706FF0B
S3150800300860601C4BDB6A13F4001F0CD0194B9B6BD2
S31508003018C3F306630133009343462A4631463846C6
S31508003028FFF7F4FEA06002B0BDE8F081114B1B68FB
S3150800303813F0040F14D00F4B1B68C3F3C1030E4FCC
S31508003048DF40A3E70B4B1B6813F4807F0AD10027E0
S315080030589CE7084B1B6813F4003F05D1002795E742
S31508003068002793E7054F91E7054F8FE74FF00008CC
S31508003078A0E700BF004402580090D00300093D00AD
S3150800308800127A002DE9F04182B0434B9B6A03F09F
S315080030980303012B69D0002B5BD0022B6CD00025CB
S315080030A800230360436083603B4B9C6AC4F3055462
S315080030B81A6CC2F30802561CDB6A13F4807F68D0C0
S315080030C8354B5F6CC7F3CC072B1C18BF0123002CA4
S315080030D808BF0023002B39D080462F4BDB6A13F430
S315080030E8800F0DD02C4B1B6CC3F34623013300937A
S315080030F83B46324621462846FFF788FEC8F80000B0
S31508003108254BDB6A13F4000F0DD0234B1B6CC3F356
S315080031180643013300933B46324621462846FFF7C5
S3150800312875FEC8F804001C4BDB6A13F0807F0DD0C7
S31508003138194B1B6CC3F30663013300933B463246AF
S3150800314821462846FFF762FEC8F8080002B0BDE81F
S31508003158F081114B1B6813F0040F14D00E4B1B6833
S31508003168C3F3C1030D4DDD409AE70B4B1B6813F4F7
S31508003178807F0AD1002593E7074B1B6813F4003FA5
S3150800318805D100258CE700258AE7054D88E7054D12
S3150800319886E7002798E700BF004402580090D00346
S315080031A800093D0000127A00154B1B6903F0380325
S315080031B8182B0ED8DFE803F00F0D0D0D0D0D0D0DAC
S315080031C8210D0D0D0D0D0D0D160D0D0D0D0D0D0DFC
S315080031D81800002070470A4B1B68C3F3C103094847
S315080031E8D84070470848704700B585B001A8FFF76A
S315080031F835FE019805B05DF804FB0448704700BF22
S31508003208004402580090D00300127A0000093D00D5
S31508003218044B9B6903F00F03034AD35C03F01F03AF
S31508003228D84070470044025874620008044BDB69AA
S31508003238C3F30213034AD35C03F01F03D84070474D
S315080032480044025874620008044BDB69C3F302237E
S31508003258034AD35C03F01F03D8407047004402585A
S315080032687462000800B585B0C2B24C4BD358020E3A
S31508003278C0F304218A401340CB4040EA0340484B38
S31508003288984228D02ED8A3F58133A3F5807398429F
S315080032985DD019D8A3F58033984248D003F5407312
S315080032A898422ED1FFF780FF3E4B9B69C3F3032351
S315080032B83D4AD35C03F01F03D840FFF7A9FFFFF781
S315080032C8C3FF05B05DF804FB384B98423FD003F5B9
S315080032D87D43984215D1334B1B6813F0005F42D1E2
S315080032E80020EEE7324B984242D00CD9314B98422F
S315080032F845D003F54073984241D0A3F580339842E8
S3150800330836D00020DDE7A3F58033984203D003F5CD
S3150800331840739842F5D1234B1B6813F0040F35D038
S31508003328204B1B68C3F3C1032348D840C9E7FFF7F6
S315080033383BFF1C4B9B69C3F303231B4AD35C03F06F
S315080033481F03D840FFF764FFFFF770FFB9E7154B6F
S315080033581B6813F0006F01D10020B2E701A8FFF738
S3150800336807FE0298ADE701A8FFF78CFE0298A8E7C2
S315080033780C4B1B6813F4807F0AD10020A1E7094B80
S315080033881B6F13F0020F05D100209AE7002098E773
S315080033980A4896E74FF4004093E700BF4C440258A2
S315080033A80803020700440258746200080803010764
S315080033B808000407080005070090D00300093D0027
S315080033C838B5036813F0010F40F08C800D460446A3
S315080033D80368454A1A408B6809690B4369690B43B0
S315080033E8E9690B4313430360EB68426822F44052C9
S315080033F813434360AB69826822F4407213438360BF
S315080034083A4B984216D03A4B98421CD0394B9842B8
S315080034181DD0394B98421ED0384B98421FD0384B8E
S31508003428984220D0374B984221D0374B984222D021
S3150800343801204EE03548FFF715FF002848D06A688E
S31508003448EAB9012045E03248FFF70CFFF5E73048AE
S31508003458FFF708FFF1E72E48FFF704FFEDE72C48CA
S31508003468FFF700FFE9E72948FFF7FCFEE5E72848E4
S31508003478FFF7F8FEE1E72648FFF7F4FEDDE72B68D5
S31508003488E9690B2B2CD8B1F5004F0DD0DBB22149D1
S3150800349851F82330B0FBF3F303EB5203B3FBF2F313
S315080034A89BB2E360002014E0DBB21A4951F82330D6
S315080034B8B0FBF3F0530803EB4000B0FBF2F34FF60A
S315080034C8F0721A40C3F342031343E360002000E096
S315080034D80120E26A22F00F022B881343E36238BD03
S315080034E80020F6E70120FAE7F369FFEF001001402C
S315080034F80044004000480040004C0040005000408E
S315080035080014014000780040007C004008030007CA
S315080035180800000784620008002301330C4A934216
S3150800352811D80269002AF8DA036943F0010303612E
S3150800353800230133064A934207D8026912F0010F9D
S31508003548F7D100207047032070470320704700BF53
S31508003558400D030084B010B5044603A880E80E00A1
S31508003568089B012B1DD1A36B23F48033A363E26860
S315080035781A4B1340E360E36823F44013E3600F9B98
S31508003588012B09D02046FFF7C7FF069B012B1BD046
S31508003598BDE8104004B07047E36843F48013E3605D
S315080035A8F0E7E36843F04003E3602046FFF7B4FF1B
S315080035B80C9B23B9A36B43F48033A363E5E7A36B9A
S315080035C823F48033A363E0E7A36843F00603A36004
S315080035D8A36843F02003A360DAE700BFBFFFBDFF77
S315080035E8022A0AD00921C26822F47052C260C36846
S315080035F843EA8123C36000207047274B0B44274AB8
S31508003608934239D9264B0B44264A934236D9264B38
S315080036180B44264A934233D9254B0B4402F5C33249
S31508003628A03293422ED9234B0B44234A93422BD9D3
S31508003638224B0B4402F5922202F57872934225D959
S315080036481F4B0B4402F5C32202F5207293421FD979
S315080036581C4B0B4402F5B71202F55872934219D956
S31508003668194B0B4402F5122202F5F862934201D966
S315080036780621B8E70721B6E70F21B4E70E21B2E716
S315080036880D21B0E70C21AEE70B21ACE70A21AAE722
S315080036980921A8E70821A6E7405327FFFF340C00AD
S315080036A8401E1BFF3F420F0000DC0BFF7F4F120036
S315080036B8808CF9FE60B6E5FE5FE3160000D3CEFE01
S315080036C8C05BB3FE00CA91FEE05459FE836843F016
S315080036D80103836000207047836823F00103836031
S315080036E80020704708B5C36823F0C043C3600129A2
S315080036F809D069B9C36843F08043C3603220FDF72F
S315080037080BFA002008BDC36843F00053C360F5E709
S315080037180120F7E7890141F02001016100230133FF
S31508003728054A934205D8026912F0200FF7D10020FE
S3150800373870470320704700BF400D0300102303613C
S3150800374800230133054A934205D8026912F0100F7F
S31508003758F7D1002070470320704700BF400D0300CB
S31508003768D0F800381943C0F8001800207047000040
S3150800377884B02DE9F041044607A880E80E002546DE
S31508003788002306E003F1400204EB8202002151609F
S3150800379801330E2BF6D9119B23BBD4F8043843F012
S315080037A80203C4F80438A36B23F40013A36323683D
S315080037B843F040032360236843F080032360002313
S315080037C8C4F8003E04F50066D4F80038C4F8003892
S315080037D80C9B012B10D1099B4BB900212046FFF7FA
S315080037E8BFFF0DE0A36B43F40013A363E7E70121CA
S315080037F82046FFF7B5FF03E003212046FFF7B0FF91
S3150800380810212046FFF786FF804608B14FF00108C9
S315080038182046FFF793FF08B14FF0010800233361EC
S315080038287361F3610AE0C3B94FF00060C2F8000992
S3150800383800220A614FF67F328A6001330799994256
S3150800384810D905EB431202F51061D2F800090028D1
S31508003858E9DB0020C2F80009EAE74FF09040C2F811
S315080038680009E5E700230AE0BBB14FF09047C2F824
S31508003878007B002202614FF67F328260013399424B
S3150800388810D905EB431202F53060D2F8007B002FF9
S31508003898EADB0027C2F8007BEBE74FF00067C2F8BF
S315080038A8007BE6E7336923F4807333610023A36159
S315080038B86FF0804363610A9B1BB9A36943F0100341
S315080038C8A361A2690A4B1343A3610D9B1BB1A369A4
S315080038D843F00803A361119B012B04D04046BDE8B9
S315080038E8F04104B07047A269024B1343A361F5E798
S315080038F800383C8004000040D0F8083813F0060366
S3150800390805D0062B18BF022B03D1022070470020CA
S3150800391870470F207047000070B40B784A78012A60
S3150800392820D0D0F81C2803F00F060124B44042EA38
S315080039380442C0F81C2800EB4310D0F8003B13F4E7
S31508003948004F0CD1D0F8002B8B68C3F30A03C9784B
S3150800395843EA81431343134A1A43C0F8002B00204D
S3150800396870BC7047D0F81C4803F00F06B24092B2F4
S315080039782243C0F81C2800EB4310D0F8002912F49B
S31508003988004FECD1D0F800498A68C2F30A02C97810
S3150800399842EA814242EA83532343024A1A43C0F859
S315080039A80029DCE70080001030B40B784A78012A31
S315080039B824D000EB4313D3F8002B002A50DBD0F8A9
S315080039C83C580A7802F00F02012404FA02F225EAA2
S315080039D80242C0F83C28D0F81C28097801F00F01E3
S315080039E88C4022EA0444C0F81C48D3F8001B234A32
S315080039F80A40C3F8002B002030BC704700EB43137D
S31508003A08D3F80029002A1EDBD0F83C580A7802F0B9
S31508003A180F02012404FA02F292B225EA0202C0F859
S31508003A283C28D0F81C28097801F00F018C40A4B26C
S31508003A3822EA0404C0F81C48D3F80019104A0A40B8
S31508003A48C3F80029D7E7D3F8002942F00062C3F87B
S31508003A580029D3F8002942F08042C3F80029D3E7A1
S31508003A68D3F8002B42F00062C3F8002BD3F8002BDA
S31508003A7842F08042C3F8002BA1E700BF0078F3EFB5
S31508003A88007833EC70B40B784C78012C24D000EB12
S31508003A98431000F530631D693E4C2C401C611D69B6
S31508003AA83D4C2C401C614C690CB18C684C611C69F6
S31508003AB844F400241C611C698D68C5F312052C435F
S31508003AC81C61012A61D0D0F8003B43F00443C0F8D2
S31508003AD8003B002070BC70474C695CBB00EB431484
S31508003AE8D4F810692C4D3540C4F81059D4F8105933
S31508003AF845F40025C4F81059D4F81069254D354001
S31508003B08C4F81059012A31D000EB4313D3F8002919
S31508003B1842F00442C3F800294B69002BD9D0D0F8E3
S31508003B283428097801F00F040121A1400A43C0F896
S31508003B383428CEE700EB431404F510642669154DBE
S31508003B48354025612669144D354025614E698D68CD
S31508003B58AE4200D94D61256945F4002525612569D8
S31508003B684E69C6F3120635432561CBE70A691AB1C9
S31508003B7800EB4311C1F8142900EB4310D0F80029CB
S31508003B8842F00442C0F80029A3E7CA68002A9AD076
S31508003B985A6198E70000F8FFFFFF07E070B49DF840
S31508003BA80C4064B903339D0807E000EB023303F5BC
S31508003BB8805351F8046B1E600134AC42F5D30020DB
S31508003BC870BC7047F0B583B00B784C78012C29D0B7
S31508003BD800EB431303F5306426697D4D35402561AE
S31508003BE826697C4D354025614D69002D40F0C18018
S31508003BF825698E68C6F3120635432561256945F495
S31508003C0800252561012A00F0C980CA78012A00F032
S31508003C18CB80D3F8002B42F00442C3F8002B0020CF
S31508003C2803B0F0BD4C6974BB00EB4314D4F81069B3
S31508003C38684D3540C4F81059D4F8105945F400258C
S31508003C48C4F81059D4F81069614D3540C4F81059AC
S31508003C58012A4AD000EB4313D3F8004944F0044438
S31508003C68C3F80049CC78012C68D04B69002BD6D00C
S31508003C78D0F83428097801F00F040121A1400A4335
S31508003C88C0F83428CBE700EB4314D4F81069504D34
S31508003C983540C4F81059D4F810694E4D3540C4F863
S31508003CA81059D4F810694D698F683D44013DB5FB34
S31508003CB8F7F5494F07EAC5453543C4F81059D4F806
S31508003CC810594E69C6F312063543C4F8105904F557
S31508003CD81064CD78012DBBD1256925F0C04525612D
S31508003CE8256945F000552561B2E70A691AB100EB5E
S31508003CF84314C4F81429CA78012A08D000EB4313D8
S31508003D08D3F8002942F00442C3F8002987E7D0F817
S31508003D18082812F4807F08D100EB4311D1F800294E
S31508003D2842F00052C1F80029E8E700EB4311D1F840
S31508003D38002942F08052C1F80029DFE7D0F8084880
S31508003D4814F4807F0ED1D3F8004944F00054C3F820
S31508003D58004914460B46C9681A789B8A0094FFF7E7
S31508003D681DFF5CE7D3F8004944F08054C3F80049BE
S31508003D78EFE78E683544013DB5FBF6F52669164F1B
S31508003D8807EAC5473E43266127698E68ADB206FB32
S31508003D9805F5C5F312053D43256133E7CA68002AC8
S31508003DA83FF433AF626130E7D0F8082812F4807F11
S31508003DB806D1D3F8002B42F00052C3F8002B28E7A7
S31508003DC8D3F8002B42F08052C3F8002B21E700BF36
S31508003DD80000F8FFFFFF07E00000F81F033292080B
S31508003DE8002393420CD210B400F58054246841F895
S31508003DF8044B01339342F7D308465DF8044B7047E2
S31508003E08084670470B784A78012A14D000EB431005
S31508003E18D0F8002B002A06DB2BB1D0F8003B23F09C
S31508003E288043C0F8003BD0F8003B43F40013C0F8C1
S31508003E38003B0020704700EB4310D0F80029002A01
S31508003E4806DB2BB1D0F8003923F08043C0F80039D7
S31508003E58D0F8003943F40013C0F80039E9E70B78BD
S31508003E684A78012A0ED000EB4310D0F8003B23F419
S31508003E780013C0F8003BCB78023BDBB2012B15D9FF
S31508003E880020704700EB4310D0F8003923F40013DC
S31508003E98C0F80039CB78023BDBB2012BF0D8D0F852
S31508003EA8003943F08053C0F80039E9E7D0F8003BF9
S31508003EB843F08053C0F8003BE2E738B505460446A8
S31508003EC8002208E004EB42134FF67F31C3F80819BD
S31508003ED8C3F8081B01320E2AF4D90022C5F810289F
S31508003EE8C5F81428C5F81C282846FFF727FC0346F2
S31508003EF808B1184638BD10212846FFF70BFC0346BB
S31508003F08F7E7D0F8003823F4FE63C0F80038D0F88D
S31508003F180038090101F4FE610B43C0F80038002097
S31508003F28704708B5D0F8043823F00203C0F80438F7
S31508003F380320FCF7F1FD002008BD08B5D0F80438C1
S31508003F4843F00203C0F804380320FCF7E5FD002017
S31508003F5808BD4269806910407047D0F8183800F5DE
S31508003F680060C0691840000C7047D0F8183800F58A
S31508003F780060C069184080B2704700EB4111D1F85B
S31508003F88082B00F5006040691040704710B4D0F857
S31508003F981048D0F8343801F00F02D340DB01DBB201
S31508003FA8234300EB411000F51060806818405DF85F
S31508003FB8044B7047406900F001007047D0F80029A3
S31508003FC8054B1340C0F80039D0F8043843F4807319
S31508003FD8C0F804380020704700F8FFFF10B4046CD6
S31508003FE8154B9C4203D9D0F8003B002B16DB00245E
S31508003FF8C0F8104BD0F8104B44F40024C0F8104B06
S31508004008D0F8104B44F01804C0F8104BD0F8104BF1
S3150800401844F0C044C0F8104B012903D000205DF8CD
S31508004028044B7047C0F8142BD0F8003B43F08023A4
S31508004038C0F8003BF2E700BF0A30544F014B18603E
S31508004048704700BF00000024C0B108B50346D0F881
S31508004058B80210B10020C3F8B802D3F8CC0210B1E0
S315080040680020C3F8CC0209B1C3F8B41218460123D4
S3150800407880F89C32027001F0C9FF08BD032070471A
S3150800408810B50446012380F89C32D0F8B83213B12B
S315080040985B6801799847D4F8CC3213B10023C4F881
S315080040A8CC32204602F024F8034608B1184610BD5B
S315080040B8204602F00DF80346F8E710B582B000234B
S315080040C8ADF8063059B10446C4F8B812CB6A0DF1F2
S315080040D806009847C4F8CC02002002B010BD032099
S315080040E8FBE708B501F0FCFF08BD08B5D0F8B832FB
S315080040F813B11B68984708BD0320FCE708B5D0F834
S31508004108B8320BB15B689847002008BD38B5044635
S3150800411800F2AA25284600F02DF90123C4F894329E
S31508004128B4F8B032C4F8983294F8AA1201F01F030A
S31508004138012B0DD03BB1022B0FD001F08001204690
S3150800414801F0F1FF03E02946204600F0CEFA38BD13
S315080041582946204600F004FBF9E72946204600F0E0
S3150800416833FBF4E710B5044629BB1346D0F8942266
S31508004178032A01D0002029E0D0F85C11D0F8602184
S3150800418891420DD8D0F8B8321B6923B190F89C2211
S31508004198032A00D19847204600F067FC002015E05E
S315080041A8891AC0F85C118A4228BF0A46194600F0DF
S315080041B854FC00200AE00A46D0F8B8329B6933B1A5
S315080041C890F89C12032904D11146984710BD03207C
S315080041D8FCE70320FAE710B50446002946D113463A
S315080041E8D0F89422022A05D094F8A032012B39D0A7
S315080041F8002046E0C269016A8A4213D88A421DD05D
S31508004208D4F8B832DB682BB194F89C22032A01D17A
S31508004218204698478021204601F085FF204600F071
S315080042282FFCE1E7521AC261194600F00EFC00237A
S315080042381A461946204601F096FFD5E7836999423A
S31508004248DED8D0F898229342DAD20022114600F036
S31508004258FCFB0021C4F898120B460A46204601F0D2
S3150800426882FFC1E7002084F8A0020AE00A46D0F8CF
S31508004278B8325B6933B190F89C12032904D1114608
S31508004288984710BD0320FCE70320FAE770B50446F3
S31508004298012380F89C320023C0F894324360C0F8A2
S315080042A8A432D0F8BC3223B1D0F8B8325B68002102
S315080042B89847402300221146204601F021FF01268F
S315080042C8A4F864614025C4F860512B460022802171
S315080042D8204601F015FFA6842562002070BD0174EA
S315080042E80020704790F89C3280F89D32042380F8A5
S315080042F89C320020704790F89C32042B01D000208D
S31508004308704790F89D3280F89C32F8E708B590F81F
S315080043189C32032B01D0002008BDD0F8B832DB69DF
S31508004328002BF8D09847F6E700207047002070471A
S315080043380020704708B5012380F89C32D0F8B832B7
S3150800434813B15B6801799847002008BD002302E08D
S315080043580133DBB201300278002AF9D118467047D2
S3150800436808B54B88012B00D008BDC0F8A43200F068
S315080043787CFBF9E70B7803704B7843708B78CA781F
S3150800438843EA022343800B794A7943EA0223838066
S315080043988B79CA7943EA0223C380704710B5044665
S315080043A8802101F0C0FE0021204601F0BCFE10BDA8
S315080043B830B583B004460D460023ADF806304A8862
S315080043C8130A013B062B00F2AB80DFE803F0041F53
S315080043D833A9A98D9A00D0F8B4321B680DF10601E5
S315080043E8007C9847EA88002A00F0A380BDF80630C2
S315080043F8002B00F099809A4228BF1A46ADF8062085
S315080044080146204600F014FB03B030BD037C43B9CF
S31508004418D0F8B8329B6A0DF1060098470223437014
S31508004428E0E7D0F8B832DB6A0DF1060098470223B0
S315080044384370D7E7D2B2052A52D8DFE802F003104C
S315080044481D2A3744D0F8B4325B6823B10DF106014A
S31508004458007C9847C6E72946FFF7A0FFD4E7D0F8B7
S31508004468B4329B6823B10DF10601007C9847B9E779
S315080044782946FFF793FFC7E7D0F8B432DB6823B1BC
S315080044880DF10601007C9847ACE72946FFF786FF39
S31508004498BAE7D0F8B4321B6923B10DF10601007CDE
S315080044A898479FE72946FFF779FFADE7D0F8B43272
S315080044B85B6923B10DF10601007C984792E7294606
S315080044C8FFF76CFFA0E7D0F8B4329B6923B10DF16A
S315080044D80601007C984785E72946FFF75FFF93E7BB
S315080044E82946FFF75BFF8FE7037C33B9D0F8B83264
S315080044F85B6B0DF10600984774E72946FFF74EFFF0
S3150800450882E7037C43B9D0F8B8321B6B0DF1060075
S3150800451898470723437065E72946FFF73FFF73E780
S315080045282946FFF73BFF6FE729462046FFF736FF80
S315080045386AE7204600F099FA66E738B504468B8894
S31508004548F3B9CB88E3B94B887F2B19D803F07F05D5
S3150800455890F89C32032B0CD080F89E52294601F01D
S31508004568F2FD204600F081FA35B1022384F89C3220
S3150800457809E0FFF713FF06E0012384F89C3202E0FE
S315080045882046FFF70BFF38BD70B504460D468978F7
S315080045982E4B197001290FD890F89C32022B11D08E
S315080045A8032B25D02946FFF7F9FE284B197820460C
S315080045B8FFF7A4FD032603E02946FFF7EFFE0326C7
S315080045C8304670BD81B14160FFF78FFD064620B1C0
S315080045D829462046FFF7E2FEF2E7204600F045FAAC
S315080045E8032384F89C32EBE700F03FFA0026E7E756
S315080045F8C9B14368994225D0D9B2FFF77FFD134B55
S31508004608197861602046FFF770FD0646B0B129465D
S315080046182046FFF7C3FE21792046FFF76FFD0223E0
S3150800462884F89C32CCE7022380F89C324160FFF775
S3150800463865FD204600F019FA0026C1E7204600F075
S3150800464814FABDE700F011FA0026B9E7EC000024D1
S3150800465808B5CB88012B0BD190F89C329BB1022B5D
S3150800466809D9032B0FD10122011D00F0E1F901E058
S31508004678FFF794FE08BD0146002341F8083F0122CA
S3150800468800F0D6F9F6E7FFF789FEF3E708B590F8DC
S315080046989C32013B022B12D8CB88022B0CD1012362
S315080046A8C360D0F8A4320BB10323C360022200F119
S315080046B80C0100F0BDF908BDFFF770FEFBE7FFF730
S315080046C86DFEF8E708B590F89C32013B022B09D82D
S315080046D84B88012B00D008BD0023C0F8A43200F08F
S315080046E8C4F9F8E7FFF75AFEF5E708B50B7803F0BB
S315080046F86003202B06D0402B04D043B1FFF74EFEAB
S31508004708002003E0D0F8B8329B68984708BD4B7874
S31508004718092B21D8DFE803F0141C201820090520E6
S31508004728100DFFF745FE0020F0E7FFF706FF00200B
S31508004738ECE7FFF729FFE9E7FFF78AFF0020E5E737
S31508004748FFF7A4FF0020E1E7FFF70AFE0020DDE7F0
S31508004758FFF7B8FF0020D9E7FFF720FE0020D5E7C6
S3150800476870B505460C460B7803F06003202B07D076
S31508004778402B05D023B1FFF711FE0026304670BD41
S3150800478895F89C32013B022B18D82379012B0FD8B0
S31508004798D5F8B8329B682146284698470646E388DE
S315080047A8002BEBD10028E9D1284600F05EF9E5E7A9
S315080047B821462846FFF7F2FD0026DFE72146284668
S315080047C8FFF7ECFD0026D9E738B505460C468A8872
S315080047D80B7803F06003202B08D0D1B2402B05D004
S315080047E85BB12146FFF7DAFD002005E0D5F8B832B7
S315080047F89B6821462846984738BD6378012B38D0E8
S31508004808002B6BD0032B40F0F08090F89C32022BDB
S3150800481806D0032B19D02146FFF7C0FD0020EBE789
S31508004828B1F1800318BF0123002908BF00233BB153
S3150800483801F079FC8021284601F075FC0020DBE7A9
S315080048482146FFF7ABFD0020D6E763884BB9B1F1DF
S31508004858800318BF0123002908BF00230BB1E3888A
S3150800486823B1284600F001F90020C5E701F05BFCF2
S31508004878F7E790F89C32022B06D0032B19D021466D
S31508004888FFF78CFD0020B7E7B1F1800318BF0123B5
S31508004898002908BF00233BB101F045FC80212846C2
S315080048A801F041FC0020A7E72146FFF777FD002025
S315080048B8A2E76388002B40F09D8011F07F0F0AD18C
S315080048C8284600F0D2F8D5F8B8329B68214628461B
S315080048D89847002090E701F02EFCF1E790F89C3203
S315080048E8022B06D0032B2FD02146FFF757FD0020B1
S315080048F882E7B1F1800318BF0123002908BF002306
S315080049089BB912F0800F15D101F07F0101EB8101E7
S315080049188B0003F5A8710144043100240C600222B7
S31508004928284600F085F8204666E72146FFF736FD53
S31508004938002061E701F07F0101EB81018B0003F19B
S31508004948100101440431E8E752B2002A24DB01F0D9
S315080049580F0303EB830398002844B0F8643153B374
S31508004968002A2EDB01F07F0202EB8202930003F590
S31508004978A8742C440434802914BF00230123002971
S3150800498808BF01233BB30023236002222146284699
S3150800499800F04EF800202FE701F00F0303EB83031E
S315080049A898002844838C002BDAD121462846FFF73D
S315080049B8F5FC002020E721462846FFF7EFFC0020F3
S315080049C81AE701F07F0202EB8202930003F1100452
S315080049D82C440434CFE7284601F054FB10B10123D0
S315080049E82360D2E700232360CFE72146FFF7D6FCEA
S315080049F8002001E70020FFE6C8B170B50D46164647
S31508004A080446FFF7A3FC01304000308028700323D2
S31508004A186B70022307E0EA5401345A1CD2B200210B
S31508004A28A9540233DBB22278002AF4D170BD704744
S31508004A3810B513460222C0F894228361C3610A4658
S31508004A48002101F088FB002010BD08B513460A4668
S31508004A58002101F080FB002008BD08B513460A4668
S31508004A68002101F080FB002008BD08B50423C0F822
S31508004A78943200231A46194601F06DFB002008BD3A
S31508004A8808B50523C0F8943200231A46194601F0DA
S31508004A986AFB002008BD72B6704762B67047000008
S31508004AA8F0B4194D2C6D24F040542C65002401E00F
S31508004AB80134E4B2112C23D8144D15F8146005EB0B
S31508004AC844056F78F51905FB00054FF4FA5CBCFB3D
S31508004AD8F5FC05FB0CF5B5F5FA5FE9D135463D4415
S31508004AE805FB000C4FF4FA55B5FBFCF50D80013DA6
S31508004AF8ADB2B5F5007FDBD216701F70012000E055
S31508004B080020F0BC704700BF00440258F062000855
S31508004B1870B58CB00022ADF82E208DF82D200CAB80
S31508004B2803F8042D0DF12D020DF12E014FF4FA703C
S31508004B38FFF7B6FF002842D0234C244B23600025F4
S31508004B48A560E560012626746574A574BDF82E303F
S31508004B586361A6619DF82D30E3619DF82C302362C8
S31508004B686662A662E66226636563A663E5632664EB
S31508004B7804236364A564E36425656365A565E6653A
S31508004B8825666566A3662046FCF75EF903950495CF
S31508004B980596069640F2676307930893099503A94D
S31508004BA82046FCF79BFA0096334602221146204611
S31508004BB8FCF7D7FA2046FCF7F0FA0CB070BDB82116
S31508004BC8034800F08BFDB7E7F000002400A000407A
S31508004BD8B462000810B58AB040F2E1730193002365
S31508004BE8029303930904049105930693079308937C
S31508004BF8522309930123024601A90E48FCF7E7FA4E
S31508004C0808B10AB010BD01210A48FCF716FB0028AE
S31508004C18F7D100F071FB00F1320401210548FCF7D1
S31508004C28FDFB0028EDD000F063FE00F065FBA0420E
S31508004C38F3D9E6E7F000002430B58BB004460D46F4
S31508004C4840211048FCF7F3FB10B900200BB030BD23
S31508004C5823466A4640210B48FCF702FB68B9009AC6
S31508004C6840F267639A4201D00020EFE7019B33B907
S31508004C789DF80E302B700120E8E70020E6E70020B3
S31508004C88E4E700BFF000002408B5FFF704FF08BDF5
S31508004C9810B500F03DFA00B910BDFBF721FB002856
S31508004CA8FAD000F0CFFDFBF793FE00F0FBFA00F010
S31508004CB833FA054B0340054A936000F02DFA446819
S31508004CC8FFF7EBFEA047E7E780FFFF1F00ED00E0D0
S31508004CD870B508E04D1C461C0B78037000F008FEFA
S31508004CE8304629462246531E9CB2002AF2D170BD88
S31508004CF838B50546002401E00134E4B20E2C12D872
S31508004D0800F0F6FD04EB44029300084AD358AB4278
S31508004D18F2D804EB44029100044A0A445268134440
S31508004D28AB42E9D900E0FF24204638BD14630008E1
S31508004D3808B5C1F3090353B903688B4209D040F88B
S31508004D48041B4FF48062FFF7C3FF012000E0002030
S31508004D5808BD0120FCE72DE9F04107460068FFF782
S31508004D68C7FFFF282CD0FCF771FB00264FF0010877
S31508004D7805E04FF00008B8F1000F1CD001361F2EC9
S31508004D8819D83D68740125443C44043400F0B0FD44
S31508004D98224629460120FCF721FC50B900231F2B7F
S31508004DA8E9D8595DE25CD2B29142E2D10133DBB26D
S31508004DB8F5E74FF00008FCF777FB4046BDE8F081B9
S31508004DC84FF00008F9E7000070B50E460E4B9842FA
S31508004DD812D004460D4B994209D10B4D2C4625B1E4
S31508004DE831462046FFF7A4FF58B1284670BDFFF79D
S31508004DF8B2FF20B12546F2E7054D2C46EFE7002518
S31508004E08EDE70025F1E700BF940500240000020835
S31508004E18900100242DE9F84305460C4617461E4618
S31508004E28DFF8848001EA08080368B3F1FF3F0AD06F
S31508004E382B6843450ED14FF00109B9F1010F12D07D
S31508004E484846BDE8F8834146FFF772FF81460028C1
S31508004E58F3D0EDE741462846FFF7B6FF0546E8B121
S31508004E684FF00109E9E72B68E41A2C44043405E0F5
S31508004E7817F8013B04F8013B013EE1D000F038FD84
S31508004E882B1DE31AB3F5806FF2D308F5806128461F
S31508004E98FFF79AFF054620B1041DE9E74FF0000918
S31508004EA8CEE74FF00009CBE700FCFFFF70B586B0E8
S31508004EB804460D4600230093884203D80E2937D89E
S31508004EC8012600E0002616B9304606B070BDFCF784
S31508004ED8BDFAAC4227D800F00BFD164963002344F7
S31508004EE89A008B188A585B68002B18BFB2F1FF3FE7
S31508004EF818D000230193202305930A46630018193E
S31508004F08810008461144497A02910244137A0393A8
S31508004F1801230493694601A8FCF730FC30B901342B
S31508004F28E4B2D6E70026FCF7BFFACDE70026FAE78B
S31508004F380026C9E7146300084FF0FF33024A1360D6
S31508004F48024A1360704700BF9001002494050024A4
S31508004F5870B504460D4616464A1E154B1B1A9A4244
S31508004F6803D9002001280CD070BDFFF7C1FEFF2821
S31508004F781AD028190138FFF7BBFEFF2816D00120DA
S31508004F88F0E70C4B23400C4A934206D02B46324690
S31508004F9821460A48FFF73EFFE6E72B4632462146F2
S31508004FA80748FFF737FFDFE70020DDE70020DBE7E4
S31508004FB8FFFF1F0800FCFFFF0000020890010024FD
S31508004FC89405002470B54A1E0F4B1B1A9A4205D938
S31508004FD8FF210E460020012812D070BD05460C4652
S31508004FE8FFF786FE064660190138FFF781FE014677
S31508004FF8FF2818BFFF2E01D00120ECE70020EAE7BA
S315080050083046FFF753FFE8E7FFFF1F08104B1B68FA
S31508005018B3F1FF3F1AD000B583B00D4A53689168BB
S315080050280B44D1680B4411690B4451690B449169C7
S315080050380B44D26913445B4202AA42F8043D042190
S315080050480448FFF785FF03B05DF804FB01207047A5
S3150800505894050024980202080D4B1B680D4A12682D
S315080050681A440D4B1B6813440C4A126813440C4A1D
S3150800507812681A440B4B1B681A440B4B1B681344DB
S315080050880A4A1268DA4201D00020704701207047A0
S315080050980000020804000208080002080C000208BA
S315080050A810000208140002081800020898020208EC
S315080050B808B50D4B1B68B3F1FF3F0BD10B4B1B68AB
S315080050C8B3F1FF3F0DD00948FFF745FE034648B13F
S315080050D8012307E00448FFF73EFE03460028EDD102
S315080050E800E00123184608BD940500249001002411
S315080050F8004870470000020808B5FFF71DFF08BDFD
S3150800510808B5FFF725FF08BD08B5FFF75BFF08BD1B
S3150800511808B5FFF7A1FF08BD08B5FFF7E9FF08BD01
S3150800512808B5FFF773FF034608B9184608BDFFF721
S31508005138BFFF0346F9E70000054BDB6913F0200FAC
S3150800514804D0034B5B6A0370012070470020704740
S315080051580048004010B5094B986200F0CDF800F1F8
S315080051680A04064BDB6913F0800F05D100F0C0FB73
S3150800517800F0C2F8A042F4D910BD00BF00480040AC
S3150800518810B588B00D4C236823F00103236000236B
S3150800519800934FF4614201920293039304930C22FD
S315080051A805920693079369462046FEF709F9236888
S315080051B843F00103236008B010BD00BF0048004053
S315080051C870B506460D46402904D82846FFF7C2FF9B
S315080051D800240BE08421074800F080FAF5E700F080
S315080051E887FB305DFFF7B6FF0134A4B2ABB2A34222
S315080051F8F5D870BDC863000870B5254B1C78BCB9CE
S315080052082448FFF799FF012801D0204670BD214B95
S315080052181B78013BDBB23F2BF7D800F06DF81E4B25
S3150800522818601E4B00221A70194B01221A70ECE7F7
S3150800523806460D46194B1B78013316481844FFF7DE
S315080052487BFF0446012815D1144B1A780132D2B2CD
S315080052581A70104B1B789A4201D00024D5E71049DA
S315080052683046FFF735FD0A4B00221A700B4B1B78A0
S315080052782B70CAE700F040F8074B1B68643398425E
S3150800528803D90024024B1C70BFE70024BDE700BF02
S31508005298D909002498090024DC090024DA0900241D
S315080052A899090024024B00221A605A609A607047CE
S315080052B810E000E008B5FFF7F5FF054B054A5A6008
S315080052C800229A6005211960034B1A6008BD00BFC1
S315080052D810E000E0FF520700E0090024044B1B68B1
S315080052E813F4803F03D0034A1368013313607047E9
S315080052F810E000E0E009002408B5FFF7EFFF014BCE
S31508005308186808BDE009002408B5FFF7F5FF08BDC9
S31508005318094B03F11801002232B19A7400225A6126
S31508005328064B054A1A6070479A745961183318313A
S315080053380132D2B2F0E700BF240A0024540A002436
S315080053480A4B1B6883B110B45C69084A146019745F
S315080053589860D86000225A74186001390844586061
S31508005368987C5DF8044B7047FF207047540A002460
S3150800537838B504460D4601281CD862002244D100D7
S31508005388114B0B445A7C1B7C9A4219D00E4B0B4482
S31508005398DA6815705A7C01325A74DA680132DA60AA
S315080053A85B689A420ED9084A084651580244D160A1
S315080053B8012038BD4FF4E171044800F08FF9DCE7A5
S315080053C80020F6E70120F4E7240A00240864000808
S315080053D808B50146024B1878FFF7CAFF08BD00BF93
S315080053E8580A002438B504460D4601281ED804EB89
S315080053F84403DA00124B13445B7CEBB16200224487
S31508005408D1000F4B0B449A6812782A705A7C013AD5
S315080054185A749A6801329A605B689A420ED9084AA1
S315080054280846515802449160012006E04FF4F2718B
S31508005438044800F053F9DAE7002038BD0120FCE7F4
S31508005448240A00240864000808B50146024B18789F
S31508005458FFF7C8FF08BD00BF9C0A002410B504461C
S31508005468012804D94FF40171044800F037F904EB10
S315080054784404E200024B1344587C10BD0864000833
S31508005488240A002438B5FFF743FF1B4C4021601C4B
S31508005498FFF756FF2070194D4021681CFFF750FF8B
S315080054A828702378FF2B1DD0FF281BD0144C002208
S315080054B814492046FEF7C8FD13492046FEF7FDFDA8
S315080054C80120FAF724FF2046FEF70BFEFDF7C4F97C
S315080054D8D4F8C402FCF7ECFF00F02CF9B0F5FA6F23
S315080054E805D338BD8521094800F0F8F8DEE74FF4FA
S315080054F8FA6000F019F9F4E7580A00249C0A00240F
S31508005508E00A00247800002414000024086400082F
S3150800551810B5064CD4F8C402FCF7E8FF2046FEF797
S31508005528AFFD0020FAF7F3FE10BD00BFE00A00241D
S3150800553870B506460D463F2906D82846FFF748FFA0
S31508005548012806D100240BE0BB210D4800F0C6F857
S31508005558F3E7BF210A4800F0C1F8F3E70134A4B21B
S31508005568ABB2A3420BD900F0C3F9305DFFF730FFA1
S315080055780128F3D0C821024800F0B0F8EEE770BD5C
S315080055880864000870B506460D461F4BD3F8C402D2
S31508005598FCF71AFD1D4B1C789CB91D48FFF754FFEC
S315080055A8012801D0204670BD194B1B78013BDBB298
S315080055B83E2BF7D8154B01221A70164B00221A7083
S315080055C8F0E7144B1B78013311481844FFF73CFFE2
S315080055D80446012801D00024E4E70E4B1A78013264
S315080055E8D2B21A700A4B1B789A4201D00024D9E71E
S315080055F809493046FFF76CFB044B00221A70054B25
S315080056081B782B70CEE700BFE00A0024F00D0024B3
S31508005618B00D0024F10D0024B10D002430B583B077
S31508005628144B1878FFF71AFF08B30546402800D91F
S315080056384025002405E09DF807200F4B1A5501342C
S31508005648E4B2A5420DD90DF107010A4B1878FFF700
S31508005658C9FE0128EFD04FF4A471084800F03EF8B7
S31508005668E9E72B46044A8121054800F074FD03B092
S3150800567830BD00BF580A0024E4090024086400085D
S31508005688E00A002470B5044600F0A8FB0646214641
S315080056980F4800F00EFD85B2002401E00134A4B2DB
S315080056A8AC420CD2315D0B4B1878FFF761FE012826
S315080056B8F4D04FF4B571084800F010F8EEE700F09A
S315080056C88DFB402302460121014800F04CFD70BDC0
S315080056D8E00A00249C0A00240864000808B500F0BB
S315080056E807F9FCE708B500F0F7F8012803D00B4BD3
S315080056F81B78012B00D008BDFFF7FEFD084B1B6879
S31508005708084A1268134403F5FA739842F3D3034B0D
S3150800571800221A70FFF7BCFAEDE700BFF80D00245F
S31508005728F40D0024FC0D0024014B1860704700BFD7
S31508005738F40D0024014B1868704700BFF40D0024C7
S3150800574808B5054B1B78012B00D008BDFFF7D4FD1B
S31508005758024B1860F9E700BFF80D0024FC0D002479
S3150800576808B5044B01221A70FFF7EAFFFFF7BAFFDC
S3150800577808BD00BFF80D002408B5FFF785FA00F044
S31508005788B3F8FFF797FDFFF7B7FC00F00DF8FFF73A
S31508005798E7FF08BD08B500F0ABF8FFF79FFD00F076
S315080057A817F8FFF79FFF08BD10B500F00FFAFFF7C7
S315080057B8AFF9064C01232370FFF7E2FC0023237098
S315080057C8FFF760FE0223237010BD00BF10000024F7
S315080057D800B583B00DF107011848FFF72DFA01281F
S315080057E810D00DF107011548FFF706FD012812D05C
S315080057F80DF107011148FFF7C5FE012814D003B0BB
S315080058085DF804FB0E4B01221A709DF807100B4829
S3150800581800F0FCF9E5E70A4B00221A709DF8071014
S31508005828064800F0F3F9E3E7054B02221A709DF8DB
S315080058380710024800F0EAF9E1E700BF000E002465
S315080058481000002408B5FFF763FE08BD38B50446FE
S315080058580D460E4B1B78012B09D00C4B1B7853B100
S315080058680A4B1B78022B0BD000F0C8F938BDC9B211
S31508005878FFF7B0F9F1E7E9B22046FFF7A1FCEFE731
S31508005888E9B22046FFF754FEEEE700BF10000024F1
S31508005898074B1B78022B05D0032B05D0012B05D007
S315080058A8402070473F2070470020704708207047FF
S315080058B810000024074B1B78022B05D0032B05D0B4
S315080058C8012B05D0402070473F20704700207047BD
S315080058D8082070471000002408B500F085F903462B
S315080058E800B10123184608BD08B5FAF707FD08BD33
S315080058F808B5FAF708FD08BD014B00225A7070472B
S31508005908400E0024034BFE22DA7018710222A3F80F
S3150800591844207047400E002410B5054C0023237018
S31508005928FFF7EAFFFF23E3700123A4F8443010BD0C
S31508005938400E0024064BFF22DA7000221A715978A5
S3150800594859719A71DA711A720622A3F844207047B7
S31508005958400E002408B50020FFF7D4FF08BD000054
S31508005968074BFF22DA70074A9A6400221A715A719D
S315080059789A710722C3F807200822A3F8442070471B
S31508005988400E002444640008044BFF22DA7042687B
S315080059989A640122A3F84420704700BF400E0024E9
S315080059A808B53120FFF7AEFF08BD000038B5084C2A
S315080059B8FF23E370002525716571FFF769FFA0715C
S315080059C8E571257265720723A4F8443038BD00BF0F
S315080059D8400E002438B5FFF78FFF0E4C01252570B9
S315080059E8FF23E3701023237100236371FFF750FF29
S315080059F8A071FFF75FFFE071FFF75CFFC0F30720B0
S31508005A0820726572A5720823A4F84430FFF774FB60
S31508005A1838BD00BF400E002438B505464478FFF760
S31508005A2837FF0138844210DC0A4C6A78A16C201DBD
S31508005A38FFF74EF9FF23E3706A78A36C1344A3644F
S31508005A486B780133A4F8443038BD2220FFF75AFF93
S31508005A58FAE700BF400E002438B504464578FFF734
S31508005A6817FF0138854211DC61680A4DA964627816
S31508005A78281DFFF72DF9FF23EB706278AB6C1344EA
S31508005A88AB6463780133A5F8443038BD2220FFF7A4
S31508005A9839FFFAE7400E0024F8B5054617460024EC
S31508005AA806E015F8013B1C44E4B2FFF721FF31462E
S31508005AB84E1E0029F5D13C600120F8BD10B5084CEA
S31508005AC8FF23E370E21D4168A06CFFF7E5FF20712C
S31508005AD800236371A3710823A4F8443010BD00BFDE
S31508005AE8400E002438B505460D4B9C6CFFF7D0FED2
S31508005AF86A1C411E2046FFF703FB60B1084CFF23CA
S31508005B08E370FFF7C5FE0138A36C0344A3640123B9
S31508005B18A4F8443038BD3120FFF7F4FEFAE700BF91
S31508005B28400E002438B504464578FFF7B1FE02381A
S31508005B3885420EDC114BFF22DA700122A3F84420B5
S31508005B48617851B9FFF7ECFA30B93120FFF7DAFE78
S31508005B5802E02220FFF7D6FE38BDA21C074B986C38
S31508005B68FFF7CEFA28B16178044A936C0B4493641C
S31508005B78F2E73120FFF7C6FEEEE700BF400E002425
S31508005B8808B54168074B986CFFF7BEFA30B1054B64
S31508005B98FF22DA700122A3F8442008BD3120FFF756
S31508005BA8B1FEFAE7400E002408B5FFF771F8034B73
S31508005BB8FF22DA700122A3F8442008BD400E00240B
S31508005BC808B589B2FFF742FE08BD0000054B00225A
S31508005BD81A709A6483F84320A3F844209A705A7076
S31508005BE8704700BF400E0024034B1B780BB10120F9
S31508005BF870470020704700BF400E0024024B002261
S31508005C0883F84320704700BF400E002408B5037880
S31508005C18FF2B04D0354A1278012A14D008BDFFF79D
S31508005C28D9FE324B93F84330012B5AD02F4BB3F990
S31508005C3844100029F2DD1846012380F84330033062
S31508005C48FFF7BEFFEAE7C93B352B46D8DFE803F07E
S31508005C583345454245453F363C394545454545451D
S31508005C6845454545454545454545454545454545CE
S31508005C7845454545454545454545241E1B21454554
S31508005C884527452A2D30FFF7C7FECAE7FFF7E4FE82
S31508005C98C7E7FFF779FEC4E7FFF710FFC1E7FFF785
S31508005CA85FFEBEE7FFF756FEBBE7FFF743FEB8E71A
S31508005CB8FFF732FEB5E7FFF715FFB2E7FFF732FF42
S31508005CC8AFE7FFF773FEACE7FFF75AFFA9E7FFF759
S31508005CD86BFFA6E7FFF764FEA3E72020FFF712FE8F
S31508005CE89FE71020FFF70EFEA0E700BF400E00242E
S31508005CF820230380004870474C0000240A230380A9
S31508005D08004870476C00002408B590F89C32032BAD
S31508005D1801D0002008BDFFF781FCFAE708B5FFF7B0
S31508005D287DFC002008BD08B50846FFF7ABFC002037
S31508005D3808BD000008B50B7813F0600F06D14B783C
S31508005D480A2B14D00B2B17D0062B01D0002008BD20
S31508005D584B881B0A212B04D00B491722FEF768FE2D
S31508005D68F4E7CA88172A28BF17220849F6E701223E
S31508005D780749FEF75DFEE9E78B7813B9044A13600D
S31508005D88E4E7FEF70BFBE1E7550000245E00002474
S31508005D988C0E002410B50446812100F0BCF90121B7
S31508005DA8204600F0B8F9002010BD000010B50446DA
S31508005DB840230222812100F0A3F94023022201216F
S31508005DC8204600F09DF94023034A0121204600F0A9
S31508005DD8CAF9002010BD00BF5813002400487047B0
S31508005DE85813002412230B80004870479400002497
S31508005DF804230B8000487047A80000240023934218
S31508005E0816D230B40BE0373401F8134000015C00B1
S31508005E18013400250D550133DBB2934206D2040F2F
S31508005E28092CF0D8303401F81340EFE730BC704736
S31508005E387047000038B50A4B186804331C680433E1
S31508005E481B68C01800D138BD064D0822A91CFFF7E3
S31508005E58D5FF042205F112012046FFF7CFFFF2E726
S31508005E6800E8F11FAC00002408B51A230B80FFF7D9
S31508005E78E1FF014808BD00BFAC00002408B50A4682
S31508005E8828B105490548FEF7B7FD034808BD024984
S31508005E980248FEF7B1FDF8E7981300247C64000869
S31508005EA810B5044C0A4621460348FEF7A5FD2046C8
S31508005EB810BD00BF981300246C64000808B50A468C
S31508005EC828B105490548FEF797FD034808BD024964
S31508005ED80248FEF791FDF8E7981300244C64000879
S31508005EE808B50A4628B105490548FEF785FD034859
S31508005EF808BD02490248FEF77FFDF8E79813002413
S31508005F085464000808B500F57171D0F80404FEF762
S31508005F18FDF808BD08B5C1EBC10293000344D3F8E0
S31508005F280822D0F80404FEF71DF908BD08B5C1EB28
S31508005F38C102930003449A6CD0F80404FEF74BF99F
S31508005F4808BD08B5D0F80404FEF7E0F908BD000056
S31508005F5810B50446C3683BB1022B0FD091210848F7
S31508005F68FFF7BCFB012100E00021D4F80404FEF782
S31508005F78B6F9D4F80404FEF789F910BD0121F4E747
S31508005F889064000810B50446D0F80404FEF7AAF988
S31508005F982268D2F8003E43F00103C2F8003E236A9D
S31508005FA823B1044A136943F006031361FAF7B0F9F3
S31508005FB810BD00BF00ED00E010B50446FAF7A9F9D0
S31508005FC8D4F80404FEF797F910BD08B5D0F8040408
S31508005FD8FEF7ACF908BD08B5D0F80404FEF7A4F92D
S31508005FE808BD10B504460120FAF791F9D4F8040457
S31508005FF8FEF79EF910BD10B504460020FAF787F992
S31508006008D4F80404FEF796F910BD000003780BB11E
S315080060180020704710B503461748C0F80434C3F87B
S31508006028C402164B0360092343600222C260002398
S31508006038036182610122C261036243628362C362A9
S315080060480363FBF72FFE80B90B4C80212046FCF72B
S31508006058E8FB402200212046FCF7BFFB80220121ED
S315080060682046FCF7BAFB002010BD4FF4937104488C
S31508006078FFF734FBE8E700BF900E0024000008404D
S3150800608890640008D0F8C43211F0800F08D101F0E6
S315080060987F01C1EBC1018A00134493F8FE017047DA
S315080060A801F07F01C1EBC1018A00134493F83E0051
S315080060B8704708B5D0F8C402FCF7E4FA08BD18B169
S315080060C8022803D003207047002070470120704734
S315080060D808B5D0F8C402FBF7BEFEFFF7F0FF08BD07
S315080060E808B5D0F8C402FBF775FEFFF7E8FF08BD48
S315080060F808B5D0F8C402FBF78EFEFFF7E0FF08BD27
S3150800610810B51C4613462246D0F8C402FCF714FA02
S31508006118FFF7D5FF10BD08B5D0F8C402FCF74DFA4D
S31508006128FFF7CDFF08BD08B5D0F8C402FCF7DDFABD
S31508006138FFF7C5FF08BD08B5D0F8C402FCF716FB7B
S31508006148FFF7BDFF08BD08B5D0F8C402FCF7E0F9AB
S31508006158FFF7B5FF08BD08B5D0F8C402FCF79BFAE7
S31508006168FFF7ADFF08BD08B5D0F8C402FCF75CFA1E
S31508006178FFF7A5FF08BD000070B50D4E0D4CA41B12
S31508006188A4100025A54209D10B4E0C4C00F02CF89A
S31508006198A41BA4100025A54205D170BD56F82530C4
S315080061A898470135EEE756F8253098470135F2E75E
S315080061B8B4640008B4640008B4640008B864000845
S315080061C810B5431E0A44914200D110BD11F8014B7F
S315080061D803F8014FF7E702440346934200D1704794
S315080061E803F8011BF9E70000F8B500BFF8BC08BCBE
S315080061F89E467047F8B500BFF8BC08BC9E4670476F
S315080062080000000000000000000000000000000078
S315080062180000000001000000020000000300000062
S31508006228040000000000000005000000000000004F
S315080062380000000000000000060000000000000042
S315080062480000000000000000070000000000000031
S3150800625801020304010203040607080900010203F0
S3150800626804050607080C1014182030400000000022
S3150800627801020304010203040607080901000000D5
S3150800628802000000040000000600000008000000E4
S315080062980A0000000C0000001000000020000000A2
S315080062A8400000008000000000010000433A2F5714
S315080062B86F726B2F736F6674776172652F4F70658F
S315080062C86E424C542F5461726765742F536F7572FA
S315080062D863652F41524D434D375F53544D3332480A
S315080062E8372F63616E2E630005020602060307034D
S315080062F80803090309040A040B040C040C050D0514
S315080063080E050F050F0610061007100800000208EC
S315080063180000020001010000000004080000020055
S315080063280201000000000608000002000301000040
S3150800633800000808000002000401000000000A081E
S31508006348000002000501000000000C080000020019
S315080063580601000000000E08000002000701000000
S3150800636800001008000002000002000000001208E1
S3150800637800000200010200000000140800000200E4
S3150800638802020000000016080000020003020000CE
S3150800639800001808000002000402000000001A089D
S315080063A8000002000502000000001C0800000200A8
S315080063B80602000000001E0800000200070200008E
S315080063C8433A2F576F726B2F736F667477617265CE
S315080063D82F4F70656E424C542F5461726765742F3F
S315080063E8536F757263652F41524D434D375F53544A
S315080063F84D333248372F72733233322E630000001A
S31508006408433A2F576F726B2F736F6674776172658D
S315080064182F4F70656E424C542F5461726765742FFE
S31508006428536F757263652F41524D434D375F535409
S315080064384D333248372F7573622E63004F70656E79
S31508006448424C540044656661756C740057696E550C
S3150800645853422042756C6B20496E74657266616397
S31508006468650000004F70656E424C5420557365727E
S315080064780000000057696E5553422042756C6B2020
S3150800648844657669636500002E2E2F5553425F448E
S3150800649845564943452F5461726765742F7573626B
S311080064A8645F636F6E662E6300000000E0
S309080064B4BD0200080F
S309080064B8990200082F
S315080064BC0090D0030090D0030100000010000000EB
S315080064CC04000000B55D00089D5D00083D5D0008F0
S315080064DC0000000000000000255D00082F5D000884
S315080064EC115D00080000000000000000000000001C
S315080064FCF95C000800000000055D00080902200090
S3150800650C010100C0320904000002FF000000070563
S3150800651C81024000FF070501024000FF0A0600023F
S3150800652C0000004001000000ED5D0008F95D000860
S3150800653CA95E0008855E0008715E0008C55E000845
S3150800654CE95E00081201000200000040501DAC6014
S3150800655C0002010203010000040309041A030000E7
S3150800656C0000000000000000000000000000000011
S30D0800657C000000000000000009
S7050800098564
